:106DB2000000B30200000301FA0400EF0500030A19
:106DC2000A5A0B001E0C00FA0D00030E00040F01FC
:106DD20064100096120132130AFA14010217010A12
:106DE2001801EF1905321A010A1B01EF1C05321FA7
:106DF200FFFF20FFFF23011E2400642A00FA2B005C
:106E0200FA2C50782D003C2E004630006432507827
:106E12003300003432FF35016436016437015038E3
:106E22000A643A00033B00043C00643E003C3F001D
:106E32000040FFFF411450420A5A430AC844053237
:106E42004500B44600FA4900024B00014C00FA50DA
:106E52000404510596520A32530B46540A965705BA
:106E620046590A465A32FA5B010A5C0A325E000A45
:106E72005F00646200FE64FFFF67FFFF6801016953
:106E820001016A05966B00006C32FF6D000473000D
:106E9200017400017801327901327E00648100645C
:106EA20084FFFF8800028A00019D0A969E00019FCE
:106EB200FFFFA0FFFFA2000AA3FFFFA40064A5003A
:106EC20064A6FFFFA7FFFFA8FFFFA9FFFF010104C0
:106ED2001501022F003C4701044803045601044EE9
:106EE200FFFF58000261FFFF6600028500AF8600C7
:106EF200018700FA89010A990008A100FAFAFAFA50
:106F02000101021501022F1E3C47010448030456E9
:106F120001034EFFFF58000261FFFF660002850079
:106F2200AF8600018700FA89010A990000A10000DA
:106F3200FAFAFA0101021501022F1E3C470102482A
:106F420003035601014EFFFF58000061FFFF660078
:106F52000085FFFF86FFFF87FFFF8901029900007E
:106F6200A10000FAFAFA0065006F00790083008D33
:106F7200009700A100AC00B600C000CA00D400DE39
:106F820000E800F20058006000680070007800809D
:106F920000880090009800A000A800B000B800C1CE
:106FA20000C800D000D800DF00E600EE00F6004185
:106FB2000047004D00530059005F0065006C0071EE
:106FC2000077007D00830089008F0095009B00A25E
:106FD20000A700AC00B200B900C000C500CA00D2D0
:0A6FE20000D500DD00E100E700EF3C
:103D750085F97485FA757E017F00E5751270FEE59B
:103D8500742FFF50010E8E5A8F5B900014E0FCA338
:103D9500E0FDEF2DFDEE3CFC8C5C8D5D900034E08C
:103DA500FAA3E0FBED2BFBEC3AFA8A5C8B5D2275FE
:103DB500A71085F97485FA757E017F00E575127087
:103DC500FEE5742FFF50010E8E5A8F5B9000DDE0EB
:103DD500B40210AC2DAD2EEF2DFDEE3CFC8C5C8DB0
:103DE5005D8016AE5AAF5B900014E0FCA3E0FDEFDA
:103DF5002DFDEE3CFC8C5C8D5DAE5CAF5D900034C2
:103E0500E0FCA3E0FDEF2DFDEE3CFC8C5C8D5D221E
:103E1500E55DF5FBE55CF5FCD29322E55DF5E9E5AD
:103E25005CF5EAD29422E55DF5EBE55CF5ECD29123
:103E350022E55DF5EDE55CF5EED2922275A710E57C
:103E45005DF5FBE55CF5FC75A700D2872275A7102B
:103E5500E55DF5E9E55CF5EA75A700D2902275A761
:103E650010E55DF5EBE55CF5EC75A700E5B54410EF
:103E7500F5B52275A710E55DF5EDE55CF5EE75A7E1
:103E850000E5B54420F5B522E50C906965F82828CC
:103E950073023F5375E700A239B34008E5B54408FE
:103EA500F5B58006E5B554F7F5B575E710023F534E
:103EB50075E700A239B34008E5B54402F5B58006BB
:103EC500E5B554FDF5B575E710023F53A23992A249
:103ED500807CA23992A1807675E700A239B34008AB
:103EE500E5B54440F5B58006E5B554BFF5B575E7CC
:103EF50010805B75E700A239B34008E5B54480F54D
:103F0500B58006E5B5547FF5B575E7108040A23953
:103F15009287803AA2399290803475E700A239B32E
:103F25004008E5B54410F5B58006E5B554EFF5B59F
:103F350075E710801975E700A239B34008E5B54467
:0E3F450020F5B58006E5B554DFF5B575E7103B
:10696500023E96023E99023EB5023ED1023ED70254
:106975003EDD023EF8023F13023F19023F1F023F70
:016985003AD7
:103F530022743490014EF0742B90014FF074329020
:103F63000150F07448900151F0746F900152F07455
:103F73006D900153F07465900154F07420900155D5
:103F8300F07434900156F07443900157F0747990B3
:103F93000158F0746C900159F0742090015AF07438
:103FA3002090015BF0742090015CF022900885E082
:103FB300FEA3E0FF741DD39F74019E400C906DB26D
:103FC300120048E493F599804C90F802E493B40509
:103FD30014900885E0FEA3E0FF906DE5120048E42D
:103FE30093F599803090F802E493D39405401490AC
:103FF3000885E0FEA3E0FF906DB2120048E493F55C
:10400300998012900885E0FEA3E0FF906E181200DD
:1040130048E493F59990088512710C900885E0FEA9
:10402300A3E0FFEFB45007EEB40103754E0022AED8
:104033005AAF5B74B48E048F05FF1270EE8C5C8DE7
:104043005DAE5AAF5B74B48E048F05FF1271198C89
:104053005A8D5BC200E55B455A601374B4C3955B2C
:10406300FFE4955AFE8E5A8F5B785C127151E574AA
:10407300A85CB80015D3955D4010E574C3955DFF4A
:10408300E4955CFE8E5C8F5D8012E5742402C3951B
:104093005DFFE4955CFE8E5C8F5DD2002290008B09
:1040A300E0B40104C20A8002D20A90008CE0B40199
:1040B30004C20B8002D20B9000C9E075F0D7A4FFB5
:1040C300AEF0740A8E048F05FF1270EE900879EC3F
:1040D300F0A3EDF09000C9E075F02BA4FFAEF090D3
:1040E3000010EEF0A3EFF07E017F00900087E01256
:1040F30070FE9000CAE08E048F05FF1270EE740A02
:10410300FF1270EE8D619000D3E075F0D7A4FFAE7F
:10411300F0740A8E048F05FF1270EE90087DECF0A8
:10412300A3EDF09000D5E060139000D5E0F5F074B6
:104133001684FF7E00EF9008DBF08006746490081D
:10414300DBF09000CBE0900065F0900117E0900069
:1041530072F0900119E0FE9000C7E08E0088F0A491
:10416300FFAEF0EF9008E4F09000F2E075F013A4D6
:10417300FDACF0900034ECF0A3EDF0A223B34016B5
:10418300900163E0700C900164E07006900165E0BB
:1041930060028002C223900163E0B4300F90016497
:1041A300E0B44708900165E0643B60028004D224D8
:1041B3008002C224900084E0FE9008E5E06E601B5C
:1041C3007599E612019C74AB90003FF01206DA7405
:1041D30064F50975080012062480FE90007CE070E7
:1041E3000674009000B1F0900069E0FE9000B1E029
:1041F300B5066390006CE0FE9000CFE0B5065790E3
:10420300006AE0FE9000DDE0B5064B900070E0FE32
:10421300900084E0B5063F90006DE0FE9000BFE0A3
:10422300B5063390006BE0FE9000CDE0B506279015
:10423300006EE0FE9000EAE0B5061B90006FE0FE22
:104243009000EBE0B5060F900071E0FE9000FDE0FA
:104253006E70030244CA90008CE070089000CDE0B9
:1042630064046002800674039000CDF0900047E080
:10427300C3940550087402900100F080149000DD8F
:10428300E060087406900100F08006740A90010053
:10429300F0900084E0B401067400900084F0900074
:1042A30084E0B4020674009000CFF0900084E0B480
:1042B300030674009000DCF09000CFE0D39401403B
:1042C30027741B900102F074009006CDF0740090E7
:1042D30006CEF07400900099F09000B1E0B40206AD
:1042E30074019000B1F080339000B1E0B4021A740D
:1042F30000900102F074009006CDF074009006CE99
:10430300F0741B900099F080127400900102F07415
:104313001B9006CDF07400900099F09000B1E0601E
:1043230014741C900098F074009006D1F0740090FF
:1043330006D2F0800C7400900098F0741C9006D1A3
:10434300F09000EAE060147419900104F074009096
:1043530006C5F074009006C6F0800C74009001044A
:10436300F074199006C5F09000EBE06014741A9095
:104373000105F074009006C9F074009006CAF0803D
:104383000C7400900105F0741A9006C9F09000FDBA
:10439300E06014742A900775F074009006C1F074FD
:1043A300009006C2F0800C7400900775F0742A9098
:1043B30006C1F09000DDE0703274059006D5F0740C
:1043C300069006D9F074079006DDF074089006E1B4
:1043D300F07400900771F07400900772F07400900D
:1043E3000773F07400900774F0804874009006D54A
:1043F300F074009006D6F074009006D9F074009023
:1044030006DAF074009006DDF074009006DEF074B6
:10441300009006E1F074009006E2F07405900771D5
:10442300F07406900772F07407900773F0740890A5
:104433000774F09000CDE0D39402401A74159007EE
:1044430065F07416900766F07417900767F0741898
:10445300900768F080277415900765F09000CDE011
:10446300B402087416900766F0800674009007661D
:10447300F07400900767F07400900768F0D2229000
:1044830000B1E0900069F09000DDE090006AF090E8
:1044930000CFE090006CF09000BFE090006DF090D2
:1044A30000CDE090006BF0900084E0900070F090FD
:1044B30000EAE090006EF09000EBE090006FF09067
:1044C30000FDE0900071F09000E7E0B40117900068
:1044D30020740FF0A374FFF0900022E4F0A3F074B3
:1044E300029000E7F09000E7E0B40341900022E07F
:1044F300FEA3E0FF900020E0FCA3E0FD12714974ED
:10450300101270FE7408120039EF9000E6F0EF709D
:104513000674FF9000E6F074009000E7F09000212D
:10452300E090009DF0900020E090009EF0900078D5
:10453300E0900075F0900077E0900074F09000A692
:10454300E0C3941E50569000A6E0F404241E90008D
:1045530076F0900076E075F0B484FF7E008F74905F
:104563000076E075F0B484ADF07C008D7590007436
:10457300E0D39575400D900074E0C3957590007479
:10458300F0800F900074E024B4C39575900074F02C
:104593000574900075E02574900075F0900075E047
:1045A30090003AF090003AE00490003BF090003A1B
:1045B300E0D39404400B90003AE0C3940490003A93
:1045C300F090003BE0D39404400B90003BE0C39495
:1045D3000490003BF0C22690003AE0D39402400DD1
:1045E30090003AE0C3940290003AF0D226C227909A
:1045F300003BE0D39402400D90003BE0C394029053
:10460300003BF0D227755E01900078E0FE9000BE7B
:10461300E0D39E5013900078E0FE9000BEE0F404D7
:104623002E0490003CF08013900078E02404FE9068
:1046330000BEE0F4042E0490003CF090003CE0D374
:104643009402400F90003CE0C3940290003CF0D2EF
:104653001D8002C21D90003CE0D39401400B9000EA
:104663003CE01490003DF0800990003CE004900091
:104673003DF012019C22C293C294C291C292C2879E
:10468300C290E5B554EFF5B5E5B554DFF5B5C2967F
:10469300C295C2A0C297C2A2C2A1E5B554BFF5B5E7
:1046A300E5B5547FF5B5E5B554FBF5B5C20C755FBB
:1046B300469000C1E07005756E028003756E037548
:1046C300550075540090000874FFF0A374DCF0C229
:1046D30011C21474C8900036F074C8900038F07595
:1046E3005300755200C204754700E570B413037597
:1046F3007000756400900016E4F0A3F0757110C2A9
:104703000FC210C20375570075560090000AE4F0FB
:10471300A3F090000CE4F0A3F0C22975590075587A
:1047230000900083E075F032A4FFAEF090001EEE1F
:10473300F0A3EFF0900073E4F09008E1E4F0C225F9
:10474300C21AD21BC21CC21DC21E90000EE4F0A3EB
:10475300F0C205C206900073E4F022755B00755A3F
:1047630000AE5AAF5B741CC39F74019E5003024892
:1047730052906DB2120048E493645F6023906DB26F
:10478300120048E493647E6017906DB2120048E40F
:10479300936481600B906DB2120048E493B4840378
:1047A300024832AE5AAF5B906DB2120048E4939068
:1047B300007712712F0FBF00010EE0FC906DB21253
:1047C3000048ECFEE493FFEEC39F5026AE5AAF5B66
:1047D3000FBF00010E906DB2120048AE5AAF5BE4FA
:1047E30093FC906DB2120048E49390007712712FFE
:1047F300ECF0AE5AAF5B906DB2120048E4939000B8
:104803007712712FE0FC906DB4120048ECFCE49336
:10481300FDECD39D4019906DB4120048E493FC90D5
:104823006DB2120048E49390007712712FECF0AE52
:104833005AAF5B74022FFF50010E8E5A8F5B785B69
:10484300740126F6500418E436F640030247642246
:10485300755B00755A00AE5AAF5B7432BE00039F9E
:104863005003024920906ECF120048E493900077E2
:1048730012712F0FBF00010EE0FC906ECF120048A3
:10488300ECFEE493FFEEC39F5026AE5AAF5B0FBF1F
:1048930000010E906ECF120048AE5AAF5BE493FC5A
:1048A300906ECF120048E49390007712712FECF0D2
:1048B300AE5AAF5B906ECF120048E493900077122C
:1048C300712FE0FC906ED1120048ECFCE493FDECF8
:1048D300D39D4019906ED1120048E493FC906ECFA3
:1048E300120048E49390007712712FECF0AE5AAFA8
:1048F3005B742D6F4E7006755B33755A00AE5AAFFD
:104903005B74022FFF50010E8E5A8F5B785B74012C
:1049130026F6500418E436F6400302485922755B24
:1049230000755A00AE5AAF5B7432BE00039F50034A
:104933000249EE906F02120048E4939000771271DF
:104943002F0FBF00010EE0FC906F02120048ECFE37
:10495300E493FFEEC39F5026AE5AAF5B0FBF000137
:104963000E906F02120048AE5AAF5BE493FC906F57
:1049730002120048E49390007712712FECF0AE5AC4
:10498300AF5B906F02120048E49390007712712F8F
:10499300E0FC906F04120048ECFCE493FDECD39D23
:1049A3004019906F04120048E493FC906F021200C8
:1049B30048E49390007712712FECF0AE5AAF5B741A
:1049C3002D6F4E7006755B33755A00AE5AAF5B742C
:1049D300022FFF50010E8E5A8F5B785B740126F60F
:1049E300500418E436F6400302492722755B00752C
:1049F3005A00AE5AAF5B7432BE00039F5003024AA3
:104A0300BC906F35120048E49390007712712F0F1A
:104A1300BF00010EE0FC906F35120048ECFEE493FA
:104A2300FFEEC39F5026AE5AAF5B0FBF00010E903F
:104A33006F35120048AE5AAF5BE493FC906F3512AA
:104A43000048E49390007712712FECF0AE5AAF5BFD
:104A5300906F35120048E49390007712712FE0FCB9
:104A6300906F37120048ECFCE493FDECD39D4019A2
:104A7300906F37120048E493FC906F35120048E4BE
:104A83009390007712712FECF0AE5AAF5B742D6FD9
:104A93004E7006755B33755A00AE5AAF5B74022FC6
:104AA300FF50010E8E5A8F5B785B740126F650041B
:104AB30018E436F640030249F52285F97485FA7540
:104AC3007E017F00E5751270FEE5742FFF50010E25
:104AD3008E5A8F5BAC5CAD5DEF2DFDEE3CFC8C5CC8
:104AE3008D5DD293D294D291D292E55DF5FBE55CD4
:104AF300F5FCE55DF5E9E55CF5EAE55DF5EBE55C1F
:104B0300F5ECE55DF5EDE55CF5EE2275A71085F9AD
:104B13007485FA757E017F00E5751270FEE5742FCA
:104B2300FF50010E8E5A8F5B7E017F769000FCE072
:104B33001270FEAC5AAD5BED2FFFEC3EFE8E5C8F28
:104B43005DE55DF5FDE55CF5FE900065E4F075A7B8
:104B5300007412900043F02285F97485FA757E0182
:104B63007F00E5751270FEE5742FFF50010E8E5A1B
:104B73008F5B900010E0FCA3E0FDEF2DFDEE3CFC0D
:104B83008C5C8D5DE55DF5FDE55CF5FE220565223A
:104B9300A2D8B34002C293A2D9B34002C294A2DA0C
:104BA300B34002C291A2DBB34002C292A2DCB34083
:104BB30030A29650067419900043F0A295500674E3
:104BC30019900043F0A2A050067419900043F0A27C
:104BD3009750067419900043F0C296C295C2A0C2C2
:104BE3009775D8402285A77375A710A2D8B3400242
:104BF300C287A2D9B34002C290A2DAB34006E5B598
:104C030054EFF5B5A2DBB34006E5B554DFF5B5A225
:104C1300DCB340089000CBE0900065F075D8408588
:104C230073A72290F800E4936406600280FE1200EA
:104C33009E75A70075D80075D90475DA0975DB0967
:104C430075DC0975DD0975DE0975D84075A7107522
:104C5300D80075D90475DA0975DB0975DC0975DDCA
:104C63000975DE0975D84075A7001200FB74C8F5F5
:104C73000975080012062475A70FE5FC900052F091
:104C8300E5FB900053F0E5FA900054F0E5F990004D
:104C930055F075A70090F800E493F52812074390A8
:104CA300088EE0D39403500790088EE0B401067495
:104CB3000090088EF090088EE09008E5F074019063
:104CC30000C0F090088EE0906986F8282873802A47
:104CD300802875A70F75F30F75A700A2A34006746C
:104CE300029000C0F0801375A70F75F31775A70026
:0A4CF300A2A4400674029000C0F075
:0C698600024CD1024CD3024CD5024CEA6A
:104CFD009000C0E0B4022AC219120AEC74029000AE
:104D0D00C0F090088EE0906992F82828738010808A
:0F4D1D000E74009000CFF0800674009000DCF060
:0C699200024D1A024D1C024D1E024D2643
:104D2C008028D219120A0174019000C0F090088EEC
:104D3C00E090699EF82828738010800E7400900013
:0A4D4C00CFF0800674009000DCF048
:0C699E00024D44024D46024D48024D508F
:104D560090F807E49390005FF090005FE0440890BD
:104D6600005FF090005FE054FE90005FF01203BD1C
:104D7600123F5490089BE0900163F090089CE090ED
:104D86000164F090089DE0900165F0900163E07089
:104D96000C900164E07006900165E060028004C238
:104DA600238002D2239000B1E004900069F09001C4
:104DB6001BE0B4FF06740090011BF090011CE0B4E8
:104DC600FF06740090011CF012475E90F802E4930F
:104DD600B40505124921801290F802E493D3940594
:104DE600400512485380031249EF74009000E7F023
:104DF6001240A0E5B54401F5B57406900045F0747F
:104E060000900046F07401900047F090F802E49399
:104E1600900048F090F803E493900049F090F8046D
:104E2600E49390004AF0740690004BF0900048E03E
:104E3600B40506740590004BF0900048E0B40406F3
:104E4600740490004BF0743090004CF074039000A2
:104E56004DF0740790004EF0740190004FF090F8FA
:104E660005E493900050F090F806E493900051F01A
:104E76007400900059F0740090005AF0740090008D
:104E86005BF0740090005CF0740090005DF07400BC
:104E960090005EF074FF900060F0A2B6B39208A294
:104EA600B3B39209A2A4B39220A2A3B39221900015
:104EB60061E4F0757000743A900777F074FD90071E
:104EC60078F0900062E4F0756F01900043E4F09092
:104ED60000C1E0B40106741A900043F0C21F756465
:104EE60000C20DD20EC203757200C2221205C6752B
:104EF6006000756C007562007566327567007568CE
:104F060000756900756A00756B00900016E4F0A3E1
:104F1600F0756D00D2B2D2A4D2B0D2B1D2A3D2A7CC
:104F2600D2A6D2A5D2B77E017F0090009EE0127075
:104F3600FE90009DE02FFF50010E900020EEF0A3A2
:104F4600EFF0EFD394FFEE940F4007900020E4F0CB
:104F5600A3F09000E6E0700674FF9000E6F0900083
:104F6600C1E07005756E028003756E0374009001D2
:104F760003F07400900106F07400900107F07429A4
:104F86009006BDF0740190076DF0740290076EF004
:104F9600740390076FF07404900770F07400900724
:104FA60069F0740090076AF0740090076BF0740063
:104FB60090076CF0D29CE571D39410400375711084
:104FC6009006BEE0D3940C400674009006BEF090A6
:104FD60006C2E0D3940C400674009006C2F0900618
:104FE600C6E0D3940C400674009006C6F09006CA3C
:104FF600E0D3940C400674009006CAF09006CEE00A
:10500600D3940C400674009006CEF09006D2E0D3FE
:10501600940C400674009006D2F09006D6E0D39425
:105026000C400674009006D6F09006DAE0D3940C95
:10503600400674009006DAF09006DEE0D3940C4049
:105046000674009006DEF09006E2E0D3940C40066B
:1050560074009006E2F0D2EC75CF01A298B3400539
:10506600C298120C54E54E6006A299B3B340028072
:1050760005C2991210E0E54F64016005E54FB404DE
:105086000280D5C28E7E087F00E5651270FEE58D32
:1050960075F008A4FDACF0EF2DFDEE3CFCE58B753C
:1050A600F02084FF7E00ED2FFFEC3EFE8E548F55E0
:1050B600D28E9000A4E0605C90001812710C9000F3
:1050C60018E0FCA3E0FD90001AE0FAA3E0FBEDB5C2
:1050D6000342ECB5023EB217A204B3401975E700CD
:1050E600A217B34008E5B54404F5B58006E5B55406
:1050F600FBF5B575E71090001AE0FEA3E0FF9000FF
:105106001CE0FCA3E0FDEF2DFDEE3CFC90001AEC4C
:10511600F0A3EDF09000B1E060099000B1E0C39417
:105126000340030251D7123027A204400890009B87
:10513600E0F546801BE560C3956150057546008025
:105146000F900088E0C3956250069000AEE0F546E9
:10515600E54675F002A4FFAEF0900883EEF0A3EFEB
:10516600F075E700AC2FAD30EDD39FEC9E402CE5FB
:10517600B5547FF5B59006BEE07006E5B554F7F573
:10518600B59000B1E0B402099000CFE0C3940240AC
:10519600028006E5B54440F5B58033900061E0C372
:1051A6009411502AE5B54480F5B59006BEE0700628
:1051B600E5B54408F5B59000B1E0B402099000CF1A
:1051C600E0C3940240028006E5B554BFF5B575E725
:1051D600109000B1E0B4032A12314275E700AE2FF9
:1051E600AF30900883E0FCA3E0FDEFD39DEE9C403A
:1051F60008E5B54480F5B58006E5B5547FF5B57587
:10520600E710A2B3300901B34041A2B3300901B39C
:105216004039A2B3300B01B34024A2B6B330070124
:10522600B34004B207800BA20CB34006740590008D
:1052360043F0A2B6B34002D21AA20BB39209A20B54
:10524600B330B301B34004A20B9209A2B6300801F1
:10525600B350030257B8A2B6300801B35003025741
:10526600B8A2B6300A01B350030256CB756F00A23E
:10527600B3B3300601B34004B206800BA20CB340B0
:10528600067405900043F0055FA205B3B35006A26D
:105296000CB3B3400302534BE56EB4032EA229B3FD
:1052A6004022E55FB40503756E01E55FC3940550C2
:1052B600069000437401F0E55FD39405400674023E
:1052C600900043F0755F01D229805EE56EB4020658
:1052D600756E01755F03E55FB40305755F0180496F
:1052E600900043E07034E55FC3940350069000439A
:1052F6007401F0E55FD3940340067402900043F016
:10530600E55FC394035002D21FE55FD394034002C6
:10531600D21FC296C295C2A0C2979000C1E0B40146
:10532600051246798003755F01C20574029008E193
:10533600F0A21D921CD21BA2A2B34002C219A21F48
:10534600B34002C21FE56EC394035006E55F6403D3
:1053560060028007B21CC21B755F01E55FB4024F95
:105366009000A4E06049900018E0FEA3E0FF9000E2
:10537600A4E08E048F05FF1270EE74018C068D0773
:1053860012003990001CEEF0A3EFF090001CE0F83C
:10539600A3E090001AC8F0A3C8F0900018E4F0A3A8
:1053A600F0C21775E700E5B554FBF5B575E710AE25
:1053B60058AF59AC54AD55EF2DFDEE3CFC8C588DD5
:1053C60059AE54AF55EFD39DEE9C401190000EE0C0
:1053D600FAA3E0FBEBC394E8EA940340028006904C
:1053E600000E12710C900008E554F0A3E555F090FC
:1053F600000AE554F0A3E555F0AE54AF5574128E8D
:10540600048F05FF1270EE8C568D57C28E758D0077
:10541600758B00756500755501755400D28E900028
:1054260008E0FEA3E0FFEF4E600B7C7A7DAC126FC6
:10543600EC8E528F53AE52AF537428BE00039F506A
:1054460010E5642FFF50010E74011200398E528F41
:10545600538553649000C8E0A852B8000DD3955305
:105466004008E553900042F080099000C8E014908F
:105476000042F0E56E60067553007552009000BF5D
:10548600E0B4040890003CE0655F6002800BA21C5B
:10549600B34004D21E8002B21E9000B1E060031237
:1054A6002CDDE570B41303757000A20D500302568F
:1054B600239000CDE0C394045006A20CB3B340037E
:1054C60002556E90007DE0B401739000FFE0B402D7
:1054D60014121281900066E075F0BCA4FFAEF08E47
:1054E6005C8F5D8056E56875F00A84FF7E00900546
:1054F60077120048E0F55B755A00AE5AAF5B900034
:10550600A2E01270FE74648E048F05FF1270EE8C9A
:105516005C8D5DE55D90003EF0AE5AAF5B90007B22
:10552600E01270FE74648E048F05FF1270EE74BC78
:105536008C068D071270FE8E5C8F5D801790007B47
:10554600E075F0BCA4FFAEF08E5C8F5D9000A2E02B
:1055560090003EF0E562C394CC5006E55D455C7074
:10556600028003124ABDD20D9000CDE0B40406902D
:1055760008E1E0700302562390007DE0B4017390C9
:1055860000FFE0B40214121281900066E075F0BCD0
:10559600A4FFAEF08E5C8F5D8056E56875F00A84D8
:1055A600FF7E00900577120048E0F55B755A00AE65
:1055B6005AAF5B9000A2E01270FE74648E048F05F1
:1055C600FF1270EE8C5C8D5DE55D90003EF0AE5A8C
:1055D600AF5B90007BE01270FE74648E048F05FF53
:1055E6001270EE74BC8C068D071270FE8E5C8F5D99
:1055F600801790007BE075F0BCA4FFAEF08E5C8F48
:105606005D9000A2E090003EF0E562C394CC5006A7
:10561600E55D455C70028003124ABDD20DE56EB4AD
:105626000106A20CB3B3400280189000CDE0B4048A
:105636000575710380097571009000447401F07559
:105646006E00E56E705B9000C4E0600D900065E052
:10565600A852B800069553400280299000C4E0B4D1
:105666000208757103756D00800CC201756D00909E
:105676000016E4F0A3F0900065E06006740990005F
:1056860043F0801D75710090003AE0B55F0690000A
:10569600447401F090003BE0B55F0674029000444C
:1056A600F0A20AB39208A2B34008900073E004F097
:1056B6008005900073E4F0900073E0B40307D20510
:1056C600900073E4F0A20AB330B601B35003025758
:1056D600B8756F0175E700E5B54401F5B575E710D6
:1056E600740B900061F0A20A9208E55FD3944740DC
:1056F60014D20CE55FD3944B400B7405900043F035
:10570600D21F755F469000CCE0B40107E56BC394E9
:105716004140028018E56BC394145008741390003E
:1057260043F08006740E900043F012467990004BC9
:10573600E0FE900048E0C39E4009900048E0D39404
:1057460008400974FB900043F0124679900049E046
:105756006015900049E0FE900047E06E600974FC19
:10576600900043F012467990004AE0601590004A96
:10577600E0FE90004CE06E600974FE900043F0126B
:10578600467990088EE060069000FCE06002800397
:10579600120BD7A2B34008900073E004F080059086
:1057A6000073E4F0900073E0B40307D20590007331
:1057B600E4F0A21FB34008C296C295C2A0C2979059
:1057C60000FCE0600CAE52AF537414BE00059F405F
:1057D600028037900084E09069AAF8282873802A0E
:1057E6008028A2A3B35005A221B340028005124B24
:1057F6000ED2218015A2A4B35005A220B340028088
:0A58060005124B0ED2208002800034
:1069AA000257E40257E60257E80257FB02580E0262
:0269BA00581073
:10581000A20FB3B3500890003CE0655F6003025BE9
:105820000BA202B35006A201B3B34003025B079080
:1058300000BFE0B404028003025AE39008E1E0B440
:1058400002028003025AD8A21EB3500302599112D9
:105850003D75900110E0601F900014E0FEA3E0FF92
:10586000900108E01270FE74C88E048F05FF12705C
:10587000EE8C5C8D5D800A900014E0F55CA3E0F591
:105880005DAE5CAF5D745E1270FE74058E048F05B4
:10589000FF1270EEAE5AAF5BED2FFFEC3EFE8E5C5A
:1058A0008F5D900034E0FCA3E0FDEF2DFDEE3CFCAD
:1058B0008C5C8D5D123E15A203B34068123DB4901E
:1058C0000110E0601F900014E0FEA3E0FF900108CB
:1058D000E01270FE74C88E048F05FF1270EE8C5CAF
:1058E0008D5D800A900014E0F55CA3E0F55DAE5C90
:1058F000AF5D745E1270FE74058E048F05FF12702A
:10590000EEAE5AAF5BED2FFFEC3EFE8E5C8F5D90EE
:105910000034E0FCA3E0FDEF2DFDEE3CFC8C5C8D43
:105920005D123E419000DDE0B40263123DB490018F
:1059300010E0D39404401BAE2DAF2E90010CE0126A
:1059400070FE74C88E048F05FF1270EE8C5C8D5D46
:105950008006852D5C852E5DAE5CAF5D745E127039
:10596000FE74058E048F05FF1270EEAE5AAF5BED2C
:105970002FFFEC3EFE8E5C8F5D900034E0FCA3E0D8
:10598000FDEF2DFDEE3CFC8C5C8D5D123E41025A1C
:10599000D6123D75900110E0D39403401F9000147F
:1059A000E0FEA3E0FF90010AE01270FE74C88E04CE
:1059B0008F05FF1270EE8C5C8D5D800A900014E004
:1059C000F55CA3E0F55DAE5CAF5D745E1270FE74D5
:1059D000058E048F05FF1270EEAE5AAF5BED2FFF00
:1059E000EC3EFE8E5C8F5D900034E0FCA3E0FDEFAA
:1059F0002DFDEE3CFC8C5C8D5D123E2BA203B34072
:105A00006B123DB4900110E0D39403401F9000143A
:105A1000E0FEA3E0FF90010AE01270FE74C88E045D
:105A20008F05FF1270EE8C5C8D5D800A900014E093
:105A3000F55CA3E0F55DAE5CAF5D745E1270FE7464
:105A4000058E048F05FF1270EEAE5AAF5BED2FFF8F
:105A5000EC3EFE8E5C8F5D900034E0FCA3E0FDEF39
:105A60002DFDEE3CFC8C5C8D5D123E639000DDE014
:105A7000B40263123DB4900110E0D39406401BAE13
:105A80002DAF2E90010EE01270FE74C88E048F05AB
:105A9000FF1270EE8C5C8D5D8006852D5C852E5D21
:105AA000AE5CAF5D745E1270FE74058E048F05FFF0
:105AB0001270EEAE5AAF5BED2FFFEC3EFE8E5C8FA8
:105AC0005D900034E0FCA3E0FDEF2DFDEE3CFC8C8E
:105AD0005C8D5D123E638009123D75123E15123ECB
:105AE0002B8024123D75123E15123E2BA203B340AB
:105AF00006123E41123E639000DDE0B40209123D01
:105B0000B4123E41123E63C20FD210A210B3B35082
:105B10000890003DE0655F6003025E0CA202B35096
:105B200006A201B3B34003025E089000BFE0B404D4
:105B3000028003025DE49008E1E0B4020280030207
:105B40005DD9A21EB35003025C92123D7590011004
:105B5000E0D39401401F900014E0FEA3E0FF900109
:105B600009E01270FE74C88E048F05FF1270EE8C6F
:105B70005C8D5D800A900014E0F55CA3E0F55DAEFD
:105B80005CAF5D745E1270FE74058E048F05FF12AB
:105B900070EEAE5AAF5BED2FFFEC3EFE8E5C8F5D7C
:105BA000900034E0FCA3E0FDEF2DFDEE3CFC8C5CAE
:105BB0008D5D123E20A203B3406B123DB4900110E4
:105BC000E0D39401401F900014E0FEA3E0FF900199
:105BD00009E01270FE74C88E048F05FF1270EE8CFF
:105BE0005C8D5D800A900014E0F55CA3E0F55DAE8D
:105BF0005CAF5D745E1270FE74058E048F05FF123B
:105C000070EEAE5AAF5BED2FFFEC3EFE8E5C8F5D0B
:105C1000900034E0FCA3E0FDEF2DFDEE3CFC8C5C3D
:105C20008D5D123E529000DDE0B40263123DB490EF
:105C30000110E0D39405401BAE2DAF2E90010DE076
:105C40001270FE74C88E048F05FF1270EE8C5C8D8E
:105C50005D8006852D5C852E5DAE5CAF5D745E1249
:105C600070FE74058E048F05FF1270EEAE5AAF5BA6
:105C7000ED2FFFEC3EFE8E5C8F5D900034E0FCA3C8
:105C8000E0FDEF2DFDEE3CFC8C5C8D5D123E520282
:105C90005DD7123D75900110E0D39403401F900032
:105CA00014E0FEA3E0FF90010BE01270FE74C88EBA
:105CB000048F05FF1270EE8C5C8D5D800A900014DD
:105CC000E0F55CA3E0F55DAE5CAF5D745E1270FE66
:105CD00074058E048F05FF1270EEAE5AAF5BED2F88
:105CE000FFEC3EFE8E5C8F5D900034E0FCA3E0FD97
:105CF000EF2DFDEE3CFC8C5C8D5D123E36A203B3B5
:105D0000406B123DB4900110E0D39403401F90000B
:105D100014E0FEA3E0FF90010BE01270FE74C88E49
:105D2000048F05FF1270EE8C5C8D5D800A9000146C
:105D3000E0F55CA3E0F55DAE5CAF5D745E1270FEF5
:105D400074058E048F05FF1270EEAE5AAF5BED2F17
:105D5000FFEC3EFE8E5C8F5D900034E0FCA3E0FD26
:105D6000EF2DFDEE3CFC8C5C8D5D123E789000DDED
:105D7000E0B40263123DB4900110E0D39407401BDD
:105D8000AE2DAF2E90010FE01270FE74C88E048FFE
:105D900005FF1270EE8C5C8D5D8006852D5C852E76
:105DA0005DAE5CAF5D745E1270FE74058E048F058F
:105DB000FF1270EEAE5AAF5BED2FFFEC3EFE8E5C35
:105DC0008F5D900034E0FCA3E0FDEF2DFDEE3CFC88
:105DD0008C5C8D5D123E788009123D75123E20125A
:105DE0003E368024123D75123E20123E36A203B389
:105DF0004006123E52123E789000DDE0B4020912D5
:105E00003DB4123E52123E78D20FC210E571906935
:095E1000BCF82828739000E4E0BE
:0369BC00025E1563
:105E1900906A2BF828287312260C801212260C80FF
:0E5E29000D122696800812274280031227428F
:0F6A2B00025E20025E25025E2A025E2F025E34AA
:105E37007571010261F812286E12298575710202C7
:105E470061F8122D21A204B340139000C9E075F048
:105E57001DA4FFAEF0900010EEF0A3EFF0900877CE
:105E6700E0FEA3E0FF740A1270FE90000AE0FCA3B4
:105E7700E0FD74098F02FF1270EE8D078C038E040C
:105E87008A058B06126FEC90087BEEF0A3EFF0907B
:105E970000CDE0B401087478BE00059F4002800D74
:105EA700747890087BF8E4F0E8A3F0801B90087BF7
:105EB700E0FEA3E0FF74F0BE00039F500B74F09068
:105EC700087BF8E4F0E8A3F0E53770037537019035
:105ED700087BE0FEA3E0FFE5372FFF50010E900897
:105EE7007BEEF0A3EFF0757103A2304015900044EC
:015EF700E0CA
:0669BF00025E3D025E498C
:105EF800906A3AF8282873800875710A80037571CA
:015F08000B8D
:096A3A00025EFF025F01025F062B
:105F09000261F89006BEE060077401F508122E4F91
:105F1900A232B3401675E700900775E0B42A06E58A
:105F2900B54402F5B575E710025FD59000B2E0D32C
:105F390094024045900086E02403A852B8000495D5
:105F4900535009900088E0D395625002800ED20226
:105F5900A22840067408900043F0D228900086E0F9
:105F6900A852B80005D39553500B900088E024033C
:105F7900C395625002C2028053900086E02403A8B0
:105F890052B8000495535010E560C39561500990CB
:105F99000088E0D395625002800ED202A228400602
:105FA9007408900043F0D228900086E0A852B80007
:105FB90005D395535014E561240FC39560400B90A8
:105FC9000088E02403C395625002C202A202400283
:105FD900C228A232B35005A202B34002801375E76A
:105FE90000900775E0B42A06E5B554FDF5B575E7E7
:105FF900109000CCE07007E56BC394144002800256
:10600900D2029000C1E0B40102D202A20240057599
:106019007104800A757110900016E4F0A3F0026112
:05602900F89000B2E058
:0669C500025F0C02602AD3
:10602E00906A43F8282873121397801212139780E0
:0E603E000D12154A8008121601800312160179
:0F6A430002603502603A02603F0260440260491F
:10604C009006C2E06006750802122E4F75710502AB
:10605C0061F812175A7571069006C6E0600675084D
:10606C0003122E4F9006CAE06006750804122E4FDC
:10607C000261F890003EE06006A204B3B3400280D7
:10608C000DE55FD39401500690003EE014F0121918
:10609C00E37571079006CEE06006750805122E4F69
:1060AC009006D2E06006750806122E4F0261F89039
:1060BC0000FFE0B40203121308121E4B7571089016
:1060CC0006D6E06006750807122E4F9006DAE060DF
:1060DC00077408F508122E4F0261F8121F2D757106
:1060EC00090261F8122305A20FB35005A210B340A8
:1060FC00028004D20FD2107571109006DEE060079A
:10610C007409F508122E4F9006E2E06007740AF548
:10611C0008122E4F0261F8900037E0C39446500AE3
:10612C00C296C2A07446900037F085375B755A0052
:10613C0090003AE0F574124032E55D900037F09033
:10614C000004E55AF0A3E55BF0C21290087BE0F581
:10615C005AA3E0F55B90003AE0F574124032E55D2D
:10616C00900036F0900000E55AF0A3E55BF0A20039
:10617C009213C2117571038073900039E0C3944679
:10618C0050139000CDE0B40102C296C295C2977430
:10619C0046900039F085375B755A0090003BE0F56E
:1061AC0074124032E55D900039F0900006E55AF02B
:1061BC00A3E55BF0C21590087BE0F55AA3E0F55B14
:1061CC0090003BE0F574124032E55D900038F090A1
:1061DC000002E55AF0A3E55BF0A2009216C214751A
:0C61EC007103800880068004800280009F
:1069CB0002605E02607F0260BB0260E70260F00261
:1069DB0061230261850261F00261F20261F40261DE
:0469EB00F60261F857
:1061F800900036E0B55F0280030262CEA211406BC8
:10620800900000E0FEA3E0FFEF4E605DAC52AD539E
:10621800740ABC0033D39D402FAA56AB5774058A25
:10622800048B05FF1270EE8D068C07900000E0FCD1
:10623800A3E0FDCFCECF1200037401120039900005
:1062480000EEF0A3EFF08021AE56AF57900000E0CB
:10625800FCA3E0FD120003740A8E048F05FF127080
:10626800EE900000ECF0A3EDF0D211AE54AF5590D3
:106278000000E0FCA3E0FDEFC39DEE9C4048124BFC
:106288005B9000CDE09069EFF82828738030D296B3
:10629800802CD2968028D296D2A08022A2134010B9
:1062A800A226301B01B34004D2A08002D296800EF1
:0E62B800A226301B01B34004D2968002D2A071
:0F69EF0002629402629602629A02629E0262A49F
:1062C600C21174C8900036F0A211B3B35007900003
:1062D60036E0B55F028048124B5B9000CDE09069D6
:1062E600FEF82828738030D296802CD2968028D249
:1062F60096D2A08022A2134010A226301B01B340E2
:1063060004D2A08002D296800EA226301B01B34092
:0763160004D2968002D2A020
:0F69FE000262EB0262ED0262F10262F50262FBDD
:10631D0074C8900036F0C211900037E0B55F02806E
:10632D00030263BFA212406B900004E0FEA3E0FFE6
:10633D00EF4E605DAC52AD53740ABC0033D39D403B
:10634D002FAA56AB5774058A048B05FF1270EE8D7C
:10635D00068C07900004E0FCA3E0FDCFCECF120029
:10636D00037401120039900004EEF0A3EFF08021C8
:10637D00AE56AF57900004E0FCA3E0FD120003748D
:10638D000A8E048F05FF1270EE900004ECF0A3ED61
:10639D00F0D212AE54AF55900004E0FCA3E0FDEF37
:1063AD00C39DEE9C400CC296C2A07446900037F07F
:1063BD00C212A212B3B35007900037E0B55F02804E
:1063CD000CC296C2A07446900037F0C212900038ED
:1063DD00E0B55F0280030264B0A214406B9000022E
:1063ED00E0FEA3E0FFEF4E605DAC52AD53740ABC0E
:1063FD000033D39D402FAA56AB5774058A048B05E5
:10640D00FF1270EE8D068C07900002E0FCA3E0FDFC
:10641D00CFCECF1200037401120039900002EEF0BE
:10642D00A3EFF08021AE56AF57900002E0FCA3E041
:10643D00FD120003740A8E048F05FF1270EE90009A
:10644D0002ECF0A3EDF0D214AE54AF55900002E083
:10645D00FCA3E0FDEFC39DEE9C4048124B5B90000A
:10646D00CDE0906A0DF82828738030D296802CD21A
:10647D00958028D295D2978022A2164010A227305F
:10648D001B01B34004D2978002D295800EA2273013
:0B649D001B01B34004D2958002D2978F
:0F6A0D0002647602647802647C0264800264860C
:1064A800C21474C8900038F0A214B3B35007900017
:1064B80038E0B55F028048124B5B9000CDE0906AEF
:1064C8001CF82828738030D296802CD2958028D248
:1064D80095D2978022A2164010A227301B01B34004
:1064E80004D2978002D295800EA227301B01B340B8
:0764F80004D2958002D29747
:0F6A1C000264CD0264CF0264D30264D70264DD4A
:1064FF0074C8900038F0C214900039E0B55F028084
:10650F00030265AAA215406B900006E0FEA3E0FF10
:10651F00EF4E605DAC52AD53740ABC0033D39D4057
:10652F002FAA56AB5774058A048B05FF1270EE8D98
:10653F00068C07900006E0FCA3E0FDCFCECF120043
:10654F00037401120039900006EEF0A3EFF08021E2
:10655F00AE56AF57900006E0FCA3E0FD12000374A7
:10656F000A8E048F05FF1270EE900006ECF0A3ED7B
:10657F00F0D215AE54AF55900006E0FCA3E0FDEF4E
:10658F00C39DEE9C40159000CDE0B40102C296C2AF
:10659F0095C2977446900039F0C215A215B3B35047
:1065AF0007900039E0B55F0280159000CDE0B4018F
:1065BF0002C296C295C2977446900039F0C21590E8
:1065CF0000CFE0B402028003026702900063E0D3C1
:1065DF0095675064900063E0F4042567FE9000D245
:1065EF00E08E00F5F0E884FF7E008F74EFC3941007
:1065FF00500CEF8574F0A4FDACF08D7480037574AE
:10660F00FF900063E0D39574400B900063E0C39557
:10661F0074F57280037572009000EDE0D3957240AF
:10662F00069000EDE0F5729000EEE0C39572500613
:10663F009000EEE0F5728071900063E0C39567FE05
:10664F009000D2E08E00F5F0E884FF7E008F74EFAB
:10665F00C39410500CEF8574F0A4FDACF08D7480D2
:10666F00037574FF85745B755A00900063E0255BBA
:10667F00FFAE5A50010E8E5A8F5B74FFBE0009D3C6
:10668F009F4005855B7280037572FF9000EDE0D32C
:10669F00957240069000EDE0F5729000EEE0C39524
:1066AF007250069000EEE0F572A204B3B3500D9055
:1066BF000064E0FE9000DAE0D39E5002801474076D
:1066CF00900043F075E700E5B554BFF5B575E710D9
:1066DF00802175A71075E700E5CDC395724008E5D9
:1066EF00B554BFF5B58006E5B54440F5B575E7106F
:1066FF0075A7009000EAE0604E9000F4E0A852B851
:10670F000004955350179000F3E0A852B8000ED331
:10671F00955340099000F5E0D395624002801575BE
:10672F00A710E5CDC394BF4004C2A28002D2A275C8
:10673F00A700801375A710E5CDC394404004C2A2F3
:10674F008002D2A275A7009000EBE0604E9000F798
:10675F00E0A852B80004955350179000F6E0A852E5
:10676F00B8000ED3955340099000F8E0D3956240DE
:10677F0002801575A710E5CDC394BF4004C2A18058
:10678F0002D2A175A700801375A710E5CDC3944061
:10679F004004C2A18002D2A175A700E570C3941373
:1067AF00501DE57075F00284AFF07E00EF4E70055E
:1067BF001232FC800AA2EDB34005C2ED1232FCAEDC
:1067CF0054AF5574B8C39F74889E400C900062E01C
:1067DF00C3945A4003026962A20CB340091246796E
:1067EF007406900043F0A20EB3500EE562D39433BB
:1067FF004007E562C394CC400280419000FFE0B4B3
:10680F000214121281900066E075F05EA4FFAEF0E4
:10681F008E5C8F5D800F90007BE075F05EA4FFAE05
:10682F00F08E5C8F5DE55D455C6011E5B54401F56B
:10683F00B5740B900061F0124ABDD20E900062E069
:10684F00D394014007E562C3941A40028002C20E3E
:10685F009006BEE060077401F508122E4F9006C235
:10686F00E060077402F508122E4F9006C6E060072D
:10687F007403F508122E4F9006CAE060077404F5F2
:10688F0008122E4F9006CEE060077405F508122E01
:10689F004F9006D2E060077406F508122E4F90064F
:1068AF00D6E060077407F508122E4F9006DAE06005
:1068BF00077408F508122E4F9006DEE06007740982
:1068CF00F508122E4F9006E2E06007740AF50812E1
:1068DF002E4F900062E0C3945A5010E570B4130924
:1068EF00900062E004F0757000803FE570B4130310
:1068FF00757000C28E758D00758B007565007555AE
:10690F0001755400D28E900061E0C394115008902D
:10691F000061E004F080067411900061F090006156
:10692F00E0B41106E5B554FEF5B5900062E0D394DE
:10693F00014007E56BC3944140028006740E90003E
:10694F0043F090088EE060069000FCE06002800348
:06695F00120BD702505E8E
:106A52000000010001400160018001A001C001E0CD
:106A620002000300039603B603D603F404000500F4
:106A72000512052405360548055A056C057E059064
:106A820005A805C005DE0600061406280646066EA1
:106A920006AE05CF06EE00FF013F015F017F019FB9
:106AA20001BF01DF01FF02FF039503B503D503F325
:106AB20003FF04FF05110523053505470559056B3D
:106AC200057D058F05A705BF05CE05F1061306272F
:106AD2000645066D06AD06ED05DD06FF0FAA0FA5FC
:106AE2000F9F0F9A0F940F8D0F870F800F780F71E2
:106AF2000F680F600F570F4E0F450F3B0F300F25DA
:106B02000F1A0F0E0F020EF50EE80EDB0ECC0EBEA4
:106B12000EAE0E9F0E8E0E7D0E6C0E5A0E470E346A
:106B22000E200E0C0DF70DE20DCB0DB50D9D0D8552
:106B32000D6D0D540D3A0D200D050CE90CCE0CB166
:106B42000C940C760C580C3A0C1B0BFB0BDB0BBB9E
:106B52000B9A0B790B570B350B130AF10ACE0AABC2
:106B62000A870A640A400A1C09F809D409B0098C88
:106B720009670943091F08FB08D608B2088E086A8C
:106B82000846082307FF07DC07B907960773075172
:106B9200072F070D06EC06CA06AA068906690649EA
:106BA200062A060A05EC05CD05B0059205750558BD
:106BB200053C0520050504EA04CF04B5049C0482C3
:106BC2000469045104390422040B03F403DE03C8EC
:106BD20003B2039D038903750361034D033B03283D
:106BE2000316030402F202E102D102C002B002A0C3
:106BF200029102820273026502570249023C022F8D
:106C020002220216020901FD01F201E601DB01D0B6
:106C120001C601BB01B101A7019D0194018B018253
:106C22000179017001680160015801500148014178
:106C320001390132012B0125011E01180111010B3D
:106C4200010500FF00FA0FA60FA00F990F920F8BFC
:106C52000F840F7C0F740F6B0F620F580F4E0F4390
:106C62000F380F2C0F1F0F120F050EF70EE80ED85C
:106C72000EC80EB70EA50E930E800E6C0E580E4265
:106C82000E2C0E150DFD0DE40DCB0DB10D950D79EC
:106C92000D5D0D3F0D200D010CE10CC00C9E0C7C16
:106CA2000C590C350C100BEA0BC40B9E0B760B4FD8
:106CB2000B260AFD0AD40AAA0A800A550A2A09FFE3
:106CC20009D409A8097C0950092508F908CD08A1A9
:106CD2000875084A081E07F307C8079D0773074986
:106CE200072006F706CE06A6067E06570630060AD7
:106CF20005E405BF059B057705540532051004EF31
:106D020004CE04AE048F047104530435041903FD48
:106D120003E203C703AD0394037B0363034B033412
:106D2200031E030802F302DE02CA02B602A30291A4
:106D3200027F026D025C024C023C022C021D020E1A
:106D4200020001F201E401D701CA01BE01B101A6AC
:106D5200019A018F0185017A01700166015D01537B
:106D6200014A0141013901310129012101190112AF
:106D7200010B010400FD00F700F000EA00E400DE70
:106D820000D900D300CE00C900C400BF00BA00B5CC
:106D920000B100AD00A800A400A0009C00990095DD
:106DA2000091008E008A008700840081007E007BB3
:10009E0075B50075840175A70075FFA075EF069004
:1000AE00003FE4F075C91075A70F75A1C775A700BD
:1000BE0075D90075CE0C75A70F75F1FE75F2FF752B
:1000CE00F30775F47875A4BA75A5FF75A60775AE16
:1000DE000075AFFF75D48175D5FF75D6FF75D7FF47
:1000EE0075A70075A20175A14775F8092275E60876
:1000FE0075E71075BC0175BE0475BD6C75BE0775D0
:10010E00BDA075BE0875BD0175BC0075BB1875BC6C
:10011E002075BA0875E88075D11375A70F75E105BE
:10012E0075E20075C7401246797597007597807411
:10013E000A1270DE7597C0E5975420700280F8752C
:10014E008F0275A700D2AF75980075A90C75A70F11
:10015E0075AB4375ADFB75AC1E75A71075C91875DB
:10016E00CA0075CB0075C80475A700758912758E07
:10017E0004758C00758A00C2A9D28C758D00758BA2
:10018E0000D2ABD28E75B62075D944C2992290009A
:10019E0079E090088DF0900084E090088EF0900049
:1001AE0085E090088FF09000A4E0900890F0900009
:1001BE00B1E0900891F09000BFE0900892F09000AE
:1001CE00CDE0900893F09000CFE0900894F090006E
:1001DE00DDE0900895F09000EAE0900896F090002F
:1001EE00EBE0900897F09000FDE0900898F09001F9
:1001FE0015E090089AF0900163E090089BF0900152
:10020E0064E090089CF0900165E090089DF09000ED
:10021E00FCE090089EF09000E6E090089FF09000C1
:10022E009DE09008A0F090009EE09008A1F0900054
:10023E0098E09008A2F0900099E09008A3F0900149
:10024E0002E09008A4F0900103E09008A5F0900160
:10025E0004E09008A6F0900105E09008A7F0900148
:10026E0006E09008A8F09006BDE09008A9F0900670
:10027E00C1E09008AAF09006C5E09008ABF0900699
:10028E00C9E09008ACF09006CDE09008ADF0900675
:10029E00D1E09008AEF09006D5E09008AFF0900651
:1002AE00D9E09008B0F09006DDE09008B1F090062D
:1002BE00E1E09008B2F0900765E09008B3F0900787
:1002CE0066E09008B4F0900767E09008B5F09007EC
:1002DE0068E09008B6F0900769E09008B7F09007D4
:1002EE006AE09008B8F090076BE09008B9F09007BC
:1002FE006CE09008BAF090076DE09008BBF09007A4
:10030E006EE09008BCF090076FE09008BDF090078B
:10031E0070E09008BEF0900771E09008BFF0900773
:10032E0072E09008C0F0900773E09008C1F090075B
:10033E0074E09008C2F0900775E09008C3F0900149
:10034E0007E09008C4F0900108E09008C5F0900115
:10035E0009E09008C6F090010AE09008C7F09001FD
:10036E000BE09008C8F090010CE09008C9F09001E5
:10037E000DE09008CAF090010EE09008CBF09001CD
:10038E000FE09008CCF0900110E09008CDF09000B6
:10039E00ABE09008CEF09000E3E09008CFF0900133
:1003AE001BE09008D0F090011CE09008D1F0229054
:1003BE00088DE0900079F090088EE0900084F09027
:1003CE00088FE0900085F0900890E09000A4F090E7
:1003DE000891E09000B1F0900892E09000BFF0908C
:1003EE000893E09000CDF0900894E09000CFF0904C
:1003FE000895E09000DDF0900896E09000EAF0900D
:10040E000897E09000EBF0900898E09000FDF090D7
:10041E00089AE0900115F090089EE09000FCF09094
:10042E00089FE09000E6F09008A0E090009DF0900C
:10043E0008A1E090009EF09008A2E0900098F09045
:10044E0008A3E0900099F09008A4E0900102F090CB
:10045E0008A5E0900103F09008A6E0900104F0904A
:10046E0008A7E0900105F09008A8E0900106F09032
:10047E0008A9E09006BDF09008AAE09006C1F090A1
:10048E0008ABE09006C5F09008ACE09006C9F0907D
:10049E0008ADE09006CDF09008AEE09006D1F09059
:1004AE0008AFE09006D5F09008B0E09006D9F09035
:1004BE0008B1E09006DDF09008B2E09006E1F09011
:1004CE0008B3E0900765F09008B4E0900766F090EE
:1004DE0008B5E0900767F09008B6E0900768F090D6
:1004EE0008B7E0900769F09008B8E090076AF090BE
:1004FE0008B9E090076BF09008BAE090076CF090A6
:10050E0008BBE090076DF09008BCE090076EF0908D
:10051E0008BDE090076FF09008BEE0900770F09075
:10052E0008BFE0900771F09008C0E0900772F0905D
:10053E0008C1E0900773F09008C2E0900774F09045
:10054E0008C3E0900775F09008C4E0900107F090A2
:10055E0008C5E0900108F09008C6E0900109F090FF
:10056E0008C7E090010AF09008C8E090010BF090E7
:10057E0008C9E090010CF09008CAE090010DF090CF
:10058E0008CBE090010EF09008CCE090010FF090B7
:10059E0008CDE0900110F09008CEE09000ABF09006
:1005AE0008CFE09000E3F09008D0E090011BF090AF
:1005BE0008D1E090011CF022754800900885E4F007
:1005CE00A3F0753200753100754E00754F00C22CC8
:1005DE00D22D90088EE06002D22274FE900887F829
:1005EE00E4F0E8A3F074FE90088BF8E4F0E8A3F0D2
:1005FE0074FE900889F8E4F0E8A3F0745A9008DFCE
:10060E00F0745A9008E0F0D22EC22AC230C22FC225
:10061E002BC232C23822750B00750A00AE0AAF0B20
:10062E00AC08AD09EDC39FEC9E401674FF1270DE50
:10063E0075CF01780B740126F6500418E436F65087
:10064E00DB22C2AF75D904758F0375B7A575B7F1E7
:10065E0090F800E4F0758F0175B7A575B7F1E52830
:10066E0090F800F075B7A575B7F190F801E4F07544
:10067E00B7A575B7F19008D3E090F802F075B7A55D
:10068E0075B7F19008D7E090F803F075B7A575B778
:10069E00F19008D4E090F804F075B7A575B7F19015
:1006AE0008D5E090F805F075B7A575B7F19008D6A6
:1006BE00E090F806F075B7A575B7F19008D8E09000
:1006CE00F807F0758F0075D944D2AF2290003FE045
:1006DE00B4AB61C2AF75D90475B62275F522758FAC
:1006EE000375B7A575B7F1740090F600F0758F011C
:1006FE00755B00755A00AE5AAF5B7445BE00279FFE
:10070E00402475B7A575B7F190088D120048E0FC2E
:10071E0090F600120048ECF0785B740126F6500457
:10072E0018E436F650D0758F0075F51175B6207534
:10073E00D944D2AF22C2AF75F52275D904755B00CC
:10074E00755A00AE5AAF5B7445BE00229F401F9093
:10075E00F600120048E493FC90088D120048ECF06D
:10076E00785B740126F6500418E436F650D575D928
:10077E004475F511D2AF2290003FE0B4AA02800377
:10078E000208C2C2AF75D90475B62275F522758FEF
:10079E000375B7A575B7F1740090F400F075B7A5A1
:1007AE0075B7F1740090F200F075B7A575B7F174D6
:1007BE000090F000F075B7A575B7F1740090EE00DB
:1007CE00F0758F01755B00755A00AE5AAF5B74FF02
:1007DE00C39F74019E402475B7A575B7F19000773D
:1007EE00120048E0FC90F400120048ECF0785B74C4
:1007FE000126F6500418E436F650CF755B00755A94
:10080E0000AE5AAF5B74FFC39F74019E402475B750
:10081E00A575B7F1900277120048E0FC90F2001235
:10082E000048ECF0785B740126F6500418E436F6B6
:10083E0050CF755B00755A00AE5AAF5B74FFC39F05
:10084E0074019E402475B7A575B7F1900477120018
:10085E0048E0FC90F000120048ECF0785B74012642
:10086E00F6500418E436F650CF755B00755A00AE9C
:10087E005AAF5B74FFC39F74019E402475B7A57574
:10088E00B7F1900677120048E0FC90EE0012004897
:10089E00ECF0785B740126F6500418E436F650CF6F
:1008AE00758F0075F51175B62075D944D2AF743AAF
:1008BE00900777F02290003FE0B4AA028003020A6C
:1008CE0000C2AF75D90475B62275F522758F037502
:1008DE00B7A575B7F1740090EC00F075B7A575B7B4
:1008EE00F1740090EA00F075B7A575B7F174009039
:1008FE00E800F075B7A575B7F1740090E600F075D5
:10090E008F01755B00755A00AE5AAF5B74FFC39FC3
:10091E0074019E402475B7A575B7F190007712004B
:10092E0048E0FC90EC00120048ECF0785B74012675
:10093E00F6500418E436F650CF755B00755A00AECB
:10094E005AAF5B74FFC39F74019E402475B7A575A3
:10095E00B7F1900277120048E0FC90EA00120048CE
:10096E00ECF0785B740126F6500418E436F650CF9E
:10097E00755B00755A00AE5AAF5B74FFC39F74016E
:10098E009E402475B7A575B7F1900477120048E024
:10099E00FC90E800120048ECF0785B740126F650EB
:1009AE000418E436F650CF755B00755A00AE5AAF98
:1009BE005B74FFC39F74019E402475B7A575B7F194
:1009CE00900677120048E0FC90E600120048ECF02A
:1009DE00785B740126F6500418E436F650CF758F06
:1009EE000075F51175B62075D944D2AF743A9007DB
:1009FE0077F022C2AF75D90475F522755B00755A72
:100A0E0000AE5AAF5B74FFC39F74019E401F90F4FB
:100A1E0000120048E493FC900077120048ECF07846
:100A2E005B740126F6500418E436F650D4755B005C
:100A3E00755A00AE5AAF5B74FFC39F74019E401F80
:100A4E0090F200120048E493FC900277120048ECFA
:100A5E00F0785B740126F6500418E436F650D4751F
:100A6E005B00755A00AE5AAF5B74FFC39F74019E54
:100A7E00401F90F000120048E493FC90047712009F
:100A8E0048ECF0785B740126F6500418E436F65004
:100A9E00D4755B00755A00AE5AAF5B74FFC39F747A
:100AAE00019E401F90EE00120048E493FC900677E2
:100ABE00120048ECF0785B740126F6500418E43608
:100ACE00F650D475F51175D944D2AF74019000C0AB
:100ADE00F0743A900777F09008E67401F022C2AFF6
:100AEE0075D90475F522755B00755A00AE5AAF5B69
:100AFE0074FFC39F74019E401F90EC00120048E4E7
:100B0E0093FC900077120048ECF0785B740126F6A7
:100B1E00500418E436F650D4755B00755A00AE5A80
:100B2E00AF5B74FFC39F74019E401F90EA001200DA
:100B3E0048E493FC900277120048ECF0785B740165
:100B4E0026F6500418E436F650D4755B00755A003C
:100B5E00AE5AAF5B74FFC39F74019E401F90E800B6
:100B6E00120048E493FC900477120048ECF0785B96
:100B7E00740126F6500418E436F650D4755B0075F1
:100B8E005A00AE5AAF5B74FFC39F74019E401F9014
:100B9E00E600120048E493FC900677120048ECF051
:100BAE00785B740126F6500418E436F650D475F5C9
:100BBE001175D944D2AF74029000C0F0743A900708
:100BCE0077F074029008E6F02274019000C0F09065
:100BDE00088EE0903CBBF828287380188016A2A3DC
:100BEE00400674029000C0F0800AA2A4400674026F
:040BFE009000C0F0B3
:0C3CBB00020BE8020BEA020BEC020BF813
:100C02009000C0E0B40105A236B34002801AD23689
:100C1200124679120A0174019000C0F01203BD124B
:100C22003F54741B900043F09000C0E0B40206A24F
:100C320036B3B34002801AC236124679120AEC74F5
:100C4200029000C0F01203BD123F54741B90004387
:100C5200F022E54F64046006E59964FF600280318A
:100C6200A22C4004D22C8027E54F600874E6254F61
:100C7200900043F0E54E600874F0254E900043F07A
:100C8200E54FB4010280FE754F00754E00C22C8004
:100C920002C22CE54F903CC7F8282873754F00E537
:100CA20099B4FF03754E01E599B4FE03754E02E552
:100CB20099B4FD03754E03E599B4FC03754E04E542
:100CC20099B4FA03754E05E599B4FB06754F011206
:100CD2004679E599B4F906754F04124679E599B457
:100CE200F733124679C29C74AB90003FF01206DAD9
:100CF20074AA90003FF09008E6E0B401051207855F
:100D020080031208C390003FE4F0D29C754F007537
:100D12004E007599F7E599D394E54007E599C39498
:100D2200F040028016859950754F027E017F00E5E2
:100D320050C394E61270FE8E338F34900885E4F02F
:100D4200A3F0E599D394C24007E599C394E6400223
:100D52008028859950754F0374E5C39550F5347515
:100D62003300AE33AF34906A521270CDE493F8740C
:100D72000193900885C8F0A3C8F0D2990210DF90C1
:100D8200089AE0700AA223B35005A224B34002805D
:100D92005C900885E0FEA3E0FF74FFBE00039F5055
:100DA20009EFC39446EE9406402B900885E0FEA31B
:100DB200E0FFEFD3946DEE94064009EFC394EEEE9C
:100DC20094064011900885E0FEA3E0FFEFD394FF64
:100DD200EE94064013900885E0FEA3E0FF900077B2
:100DE200120048E599F08003859975801190088575
:100DF200E0FEA3E0FF900077120048E599F090082A
:100E02008512710C900885E0FEA3E0FFEFB40106A5
:100E1200EEB407028003020EDA900777E0B43C02D8
:100E22008003020EDAA223B35005A224B34002804B
:100E320055C29C1203BD900084E09008E5F0124078
:100E4200A0900163E090089BF0900164E090089C00
:100E5200F0900165E090089DF074AB90003FF012B5
:100E620006DA74AA90003FF09008E6E0B401051299
:100E7200078580031208C39008E6E09000C0F09056
:100E8200003FE4F08047C29C12019C740090089BD2
:100E9200F0740090089CF0740090089DF09000841B
:100EA200E09008E5F01240A074AB90003FF012060B
:100EB200DA74AA90003FF01207851208C3D29C751B
:100EC20099FB75096475080012062480FED29C7590
:100ED2004F00754E007599FB0210DF900885E0FE09
:100EE200A3E0FFEF4E7006859932753100900885B8
:100EF200E0FEA3E0FF74016F4E701BAC31AD32AA6D
:100F020033AB34ED2BFBEC3AFA8A068B0790007771
:100F1200120048E599F090088512710C900885E05E
:100F2200FEA3E0FF74026F4E7021AC31AD327456F5
:100F32006D4C7006E55064E6600280031246791239
:100F420040A0855099754F00754E000210DF900841
:100F520085E0FEA3E0FF900077120048E599F0904B
:100F6200088512710C900885E0FEA3E0FFAC33AD5A
:100F7200348F028E038C068D07906A981270CDE42E
:100F820093F9740193FEEAD39EEB99400985509937
:100F9200754F00754E000210DF900885E0FEA3E059
:100FA200FF900077120048E599F090088512710CC5
:100FB200900885E0FEA3E0FFEFB40006EEB4010264
:100FC20080030210DF900055E0D394C7400B9000DD
:100FD20055E0C394C8F551801A900055E0D394634C
:100FE200400B900055E0C39464F551800690005583
:100FF200E0F551E55175F002A4FFAEF08F74EF9069
:10100200007712712FEFFCE0FDEC90007A12712F45
:10101200EDFCE0FDEC2DB5510280030210D10FEF83
:1010220090007712712FE574FFE0FCEF90007B12C5
:10103200712FECFFE0FCEFC39CB55102800302105C
:10104200D1E57490007912712FE574FFE0FCEF9006
:10105200007C12712FECFFE0FCEF2CB55171E574AE
:1010620090007D12712FE0C395519008D3F0E57482
:1010720090007E12712FE0C395519008D4F0E57470
:1010820090008112712FE0C395519008D5F0E5745C
:1010920090008212712FE0C395519008D6F0E5744A
:1010A20090008312712FE0C395519008D7F0E57438
:1010B20090008412712FE0C395519008D8F0120667
:1010C200507599F975096475080012062480FE7539
:0D10D20099FF75096475080012062480FE60
:0F3CC700020C9E020D81020EDD020F50020F9BB8
:1010DF0022E54E903CD6F82828730211C49008855B
:1010EF00E0FEA3E0FF900045120048E0F59990085C
:1010FF008512710C900885E0FEA3E0FF741C6F4E03
:10110F007003754E000211C4856F990211C49008C7
:10111F0085E0FEA3E0FF900077120048E0F599EF1D
:10112F00B40107EEB40703754E0090088512710CD9
:07113F000211C4900886E0D4
:0F3CD6000210E90210EC02111702111D02114237
:10114600903D48F828287385539980678560998073
:1011560062856299805D8566998058856899805315
:10116600856999804E856A998049856B99804490F6
:101176000017E0F599803CA22DB340077599FAC295
:101186002D8017A222B3400575990F800B9000435E
:10119600E0F599900043E4F0C2228017856C9980AF
:1011A60012856799800D856D9980087599FC800375
:0311B600754E0073
:103D480002114D02115202115702115C0211610257
:103D5800116602116B02117002117502117D0211B8
:0D3D6800A20211A70211AC0211B10211B6A6
:0B11B90090088512710C8003123FAFFC
:033CE5000211C108
:1011C40022E538255BFFAE5A50010E9000771200DD
:1011D40048E0F539E538255BFFAE5A50010E0FBFE4
:1011E40000010E900077120048E0F53A85403CE596
:1011F40039B53A058539388041E53AD39539401DEA
:10120400E53AC39539853BF0A4FFAEF0E53C8E0486
:101214008F05FF1270EEED2539F538801DE539C3D1
:10122400953A853BF0A4FFAEF0E53C8E048F05FFB4
:101234001270EEEDF4042539F53822E53AD39539E8
:10124400401DE53AC39539853BF0A4FFAEF0E53C7B
:101254008E048F05FF1270EEED2539F538801DE5FB
:1012640039C3953A853BF0A4FFAEF0E53C8E048F7C
:1012740005FF1270EEEDF4042539F5382290007D57
:10128400E0B4017FE56875F00A84FF7E008F38E5DD
:101294006875F00A84ADF07C008D3B75400A755A80
:1012A40005755B24E538C3941150051211C58006F9
:1012B4009005ACE0F538E538C394F05008E5389073
:1012C4000066F0800674EF900066F0E56875F00A39
:1012D40084FF7E008F38E56875F00A84ADF07C00E9
:1012E4008D3B75400A755A05755B5AE538C39411F0
:1012F40050051211C580069005E2E0F538E53890F6
:10130400003EF02290007DE0B401028003021396B7
:10131400E56875F00A84FF7E008F38E56875F00A89
:1013240084ADF07C008D3B75400A755A05755B36BB
:10133400E538C3941150051211C580069005BEE02E
:10134400F538E538C394F0500585384C8003754C66
:10135400EFE56875F00A84FF7E008F38E56875F064
:101364000A84ADF07C008D3B75400A755A05755BA7
:1013740048E538C3941150051211C580069005D074
:10138400E0F538E538C394F0500585384D80037591
:101394004DEF22E56075F00484FF7E008F38E56030
:1013A40075F00484ADF07C008D3B754004755A01E2
:1013B400755B00E538C3943F50051211C580069053
:1013C40001B6E0F538E53890087FF8E4F0E8A3F0DA
:1013D400900042E075F020A4FFAEF09000C8E08ECB
:1013E400048F05FF1270EE8D389000B0E0D3956045
:1013F40050030214A29000D4E0D395604010ED9005
:1014040001B712712FE0F52C752B0002149F900088
:101414009FE0D395604043E5389001B712712FE007
:10142400F539E5389001D712712FE0F53A9000D4E0
:10143400E0F4042560F53B90009FE0FE9000D4E0CA
:10144400F4042EF53CE539B53A05853938800312A4
:10145400123F85382C752B008041E5389001D71256
:10146400712FE0F539E5389001F712712FE0F53A64
:1014740090009FE0F4042560F53B9000B0E0FE90FE
:10148400009FE0F4042EF53CE539B53A058539387A
:10149400800312123F85382C752B000215499000E9
:1014A400D7E0D395605011E53890023712712FE0E0
:1014B400F52C752B000215499000A0E0D3956050DF
:1014C40043E53890021712712FE0F539E5389002A0
:1014D4003712712FE0F53A9000A0E0F4042560F58E
:1014E4003B9000D7E0FE9000A0E0F4042EF53CE52C
:1014F40039B53A05853938800312123F85382C7581
:101504002B008041E5389001F712712FE0F539E5A1
:101514003890021712712FE0F53A9000B0E0F4040D
:101524002560F53B9000A0E0FE9000B0E0F4042EAE
:10153400F53CE539B53A05853938800312123F8503
:10154400382C752B00229000E8E0F53D75401175AC
:101554005A02755B00AE52AF53E53D75F00FA4FD22
:10156400ACF0EDD39FEC9E4021E53D8E048F05FF4A
:101574001270EEED75F010A4FFAEF0E56075F01199
:1015840084FD7C00ED2FF53E800EE56075F011843E
:10159400FF7E00EF24F0F53E853E38E56075F011DE
:1015A40084AFF07E008F3B1211C585383FAE52AF39
:1015B400539000E8E075F00FA4FDACF0EDD39FEC80
:1015C4009E4028755A02755B10853E381211C585F8
:1015D4003F3985383AAE52AF53E53D8E048F05FF4F
:1015E4001271198D3B853D3C12123FE53890087FFE
:1015F400F8E4F0E8A3F0752C64752B00229000E861
:10160400E0F53D754011755A02755B00AE52AF535B
:10161400E53D75F00FA4FDACF0EDD39FEC9E4021A9
:10162400E53D8E048F05FF1270EEED75F010A4FFFA
:10163400AEF0E56275F01184FD7C00ED2FF53E807F
:101644000EE56275F01184FF7E00EF24F0F53E850F
:101654003E38E56275F01184AFF07E008F3B1211C5
:10166400C585383FAE52AF539000E8E075F00FA443
:10167400FDACF0EDD39FEC9E4028755A02755B10CB
:10168400853E381211C5853F3985383AAE52AF537D
:10169400E53D8E048F05FF1271198D3B853D3C128B
:1016A400123FE53890087FF8E4F0E8A3F0E56C60B9
:1016B40017E56CC394FE50109000DCE0B40209906E
:1016C40000CAE0D3940B5002801F90087FE0FEA371
:1016D400E0FFE56C1270FE74E78E048F05FF127054
:1016E400EE90087FECF0A3EDF09000B2E0B4045F5C
:1016F400E56075F00484FF7E008F38E56075F004C2
:1017040084ADF07C008D3B754004755A01755B0017
:10171400E538C3943F50051211C580069001B6E028
:10172400F53890087FE0FEA3E0FFE5381270FE7400
:10173400328E048F05FF1270EE90087FE0FEA3E066
:10174400FFEF2DFDEE3CFC90087FECF0A3EDF0756F
:101754002C64752B002290007DE0B40146E5687589
:10176400F00A84FF7E008F38E56875F00A84ADF0D6
:101774007C008D3B75400A755A05755B00E538C3DE
:10178400941150051211C58006900588E0F538AE15
:101794002BAF2CE5382FFF50010E74641271418E6B
:1017A4002B8F2C90007EE0B40146E56975F00A8425
:1017B400FF7E008F38E56975F00A84ADF07C008DFA
:1017C4003B75400A755A05755B6CE538C394115036
:1017D400051211C580069005F4E0F538AE2BAF2C48
:1017E400E5382FFF50010E74641271418E2B8F2C3B
:1017F40090008DE0B40249E56BC3944175F0058413
:10180400FF7E008F38E56B75F00584ADF07C008DAC
:101814003B754005755A06755B00E538C394135053
:10182400051211C5800690068AE0F538AE2BAF2C60
:10183400E5382FFF50010E74641271418E2B8F2CEA
:101844009000CFE0B4020280030218F9E56075F05D
:101854001584FF7E008F38E56075F01584ADF07C4B
:10186400008D3B754015755A03755BF4E538C394D8
:101874000B50051211C58006900476E0F538E53862
:1018840075F0FFA4FFAEF09000D0E08E048F05FF4A
:101894001270EEED900063F0E56775F078A4FFAE8A
:1018A400F074FF8E048F05FF1270EE8C5A8D5B74FA
:1018B400028C068D071200398F38AC5AAD5B740464
:1018C400FF1271198D3B754004755A06755B28E546
:1018D40038C3941D50051211C580069006BCE0F56E
:1018E40038AE2BAF2CE5382FFF50010E7464127103
:1018F400418E2B8F2C90007CE0B4025DE56275F084
:1019040064A4FFAEF074081200398E5C8F5D740518
:101914008E048F05FF1270EE8D38AE5CAF5D7405DA
:101924008E048F05FF1271198D3B754005755A059C
:10193400755BDEE538C3941350051211C58006901B
:101944000668E0F538AE2BAF2CE5382FFF50010EBA
:1019540074641271418E2B8F2C9000BEE0707F90C6
:101964000042E075F00A84FF7E008F38900042E068
:1019740075F00A84ADF07C008D3B75400A755A05FC
:10198400755BC0E538C3940E50051211C5800690EE
:101994000645E0F538E538900067F09000DDE0B4E6
:1019A400023C900042E075F00A84FF7E008F38907C
:1019B4000042E075F00A84ADF07C008D3B75400A6E
:1019C400755A05755BCFE538C3940E50051211C5E1
:1019D4008006900654E0F538E538900068F02290CF
:1019E4000085E0B401179008DAE0252CFFAE2B50F7
:1019F400010E9000D9E01271418E2B8F2C9000FDC6
:101A0400E0B401149000FEE0A852B80004955350CD
:101A140007E560C39561400280139000A7E0252C80
:101A2400FFAE2B50010E8E2B8F2C021E4A90008588
:101A3400E0B40306A22AB3B3400280509008E4E065
:101A440070109008DDE0C39405A852B800069553C1
:101A5400400280109000A7E0252CFFAE2B50010E11
:101A64008E2B8F2C9008E4E0600D9008DDE0A852E6
:101A7400B800069553400280109000A7E0252CFF83
:101A8400AE2B50010E8E2B8F2C021E4A90007FE04D
:101A9400B402028003021E4A900082E0602FE568CF
:101AA400D39446402890000EE0FEA3E0FF9000BDD2
:101AB400E075F003A4FDACF0EFD39DEE9C400E90D6
:101AC40000E1E0A852B80005D395535003021E4A22
:101AD4009000B2E0B403028003021C9285625B753D
:101AE4005A00900089E0A852B800049553500E9013
:101AF400008AE0A85AB80005D3955B5003021C8FF6
:101B0400E56275F002A4FFAEF074158E048F05FF34
:101B14001270EE8C068D07900607120048FEE0FF57
:101B2400EE900081E0FEEF8E0088F0A4FFAEF0742A
:101B3400648E048F05FF1270EE8C5A8D5B90004208
:101B4400E075F018A4FFAEF09000C8E08E048F0595
:101B5400FF1270EE8C068D0790061F120048AE5AD5
:101B6400AF5BE01270FE74648E048F05FF1270EE9A
:101B74008C5A8D5BE566A85AB80005D3955B500373
:101B8400021C06E566C3955BFFE4955AFE8E5A8FE8
:101B94005B7428BE00039F500C755B28755A007453
:101BA4000D900043F0AE5AAF5B900082E01270FEDD
:101BB40074288E048F05FF1270EE8C5A8D5B90088A
:101BC4007FE0FEA3E0FF740A8E048F05FF1270EE1F
:101BD4008D068C07AC5AAD5BCFCECF120003740ACE
:101BE4008E048F05FF1270EE8C5A8D5B90087FE097
:101BF400FEA3E0FF12714990087FEEF0A3EFF0021C
:101C04001C8FE566A85AB80004955B507EAE5AAFA7
:101C14005BE5661271418E5A8F5B7428BE00039F88
:101C2400500C755B28755A00740D900043F0AE5A41
:101C3400AF5B900082E01270FE74288E048F05FF63
:101C44001270EE8C5A8D5B90087FE0FEA3E0FF7467
:101C54000A8E048F05FF1270EE8D068C07AC5AAD08
:101C64005BCFCECF120003740A8E048F05FF12706F
:101C7400EE8C5A8D5B90087FE0FEA3E0FFEF2DFD14
:101C8400EE3CFC90087FECF0A3EDF0021E4A9000BD
:101C9400CAE08560F0A4FFAEF074051270FE74070C
:101CA4001200398E5A8F5B900089E0A852B8000464
:101CB4009553501290008AE075F002A4FDACF0EF49
:101CC400C39DEE9C4003021E4AE56075F00B84FF41
:101CD4007E00900607120048FEE0FFEE900081E0CF
:101CE400FEEF8E0088F0A4FFAEF074648E048F05BE
:101CF400FF1270EE8C5A8D5B900042E075F018A4D0
:101D0400FFAEF09000C8E08E048F05FF1270EE8CD9
:101D1400068D0790061F120048AE5AAF5BE01270A2
:101D2400FE74648E048F05FF1270EE8C5A8D5BE591
:101D340066A85AB80005D3955B5003021DC1E56639
:101D4400C3955BFFE4955AFE8E5A8F5B7428BE00E0
:101D5400039F500C755B28755A00740D900043F076
:101D6400AE5AAF5B900082E01270FE74288E048F2E
:101D740005FF1270EE8C5A8D5B90087FE0FEA3E0A5
:101D8400FF740A8E048F05FF1270EE8D068C07AC6B
:101D94005AAD5BCFCECF120003740A8E048F05FFB9
:101DA4001270EE8C5A8D5B90087FE0FEA3E0FF1268
:101DB400714990087FEEF0A3EFF0021E4AE566A891
:101DC4005AB80004955B507EAE5AAF5BE56612715B
:101DD400418E5A8F5B7428BE00039F500C755B289C
:101DE400755A00740D900043F0AE5AAF5B900082B8
:101DF400E01270FE74288E048F05FF1270EE8C5A68
:101E04008D5B90087FE0FEA3E0FF740A8E048F05CB
:101E1400FF1270EE8D068C07AC5AAD5BCFCECF129D
:101E24000003740A8E048F05FF1270EE8C5A8D5BCA
:101E340090087FE0FEA3E0FFEF2DFDEE3CFC900850
:101E44007FECF0A3EDF0229000DDE0B4027BE560CE
:101E540075F00884FF7E008F38E56075F00884AD66
:101E6400F07C008D3B754008755A01755BE0E538E0
:101E7400C3943F50051211C58006900276E0F538F0
:101E8400E538900881F8E4F0E8A3F0900881E0FEDA
:101E9400A3E0FFAC2BAD2C12000374648E048F05F9
:101EA400FF1270EE900881ECF0A3EDF090007AE060
:101EB4008C068D071270FE74648E048F05FF1270F9
:101EC400EE900881ECF0A3EDF090087FE0FEA3E033
:101ED400FFAC2BAD2C12000374648E048F05FF122B
:101EE40070EE90087FECF0A3EDF090007AE08C06A1
:101EF4008D071270FE74648E048F05FF1270EE90CD
:101F0400087FECF0A3EDF0A204401DAE52AF537471
:101F140005BE00039F5002D204E562D394CC40086E
:101F2400D2027411900043F0229000DCE0B4020865
:101F34009000CAE0640B6002804590087FE0FEA335
:101F4400E0FFE56C1270FE74E78E048F05FF1270DB
:101F5400EE90087FECF0A3EDF09000DDE0B4021FFA
:101F6400900881E0FEA3E0FFE56C1270FE74E78E3A
:101F7400048F05FF1270EE900881ECF0A3EDF09051
:101F8400009CE05402601B900093E0A852B8001239
:101F9400D39553400DA204B3B35007E562C3949A9A
:101FA4004002805FAE35AF36900091E075F002A438
:101FB400FDACF0EF2DFDEE3CFC74022DFD50010C48
:101FC400E562BC003ED39D403A754401A2314033E2
:101FD400900092E075F05EA4FDACF07405FF127001
:101FE400EE8C5C8D5D124ABD90087FE0FEA3E0FF9D
:101FF400900092E02FFF50010E90087FEEF0A3EFC7
:10200400F0D231E562A835B8000495365002C231E9
:10201400856236753500E54470030221239000EF94
:10202400E0C3954450030221159000FFE0C39402DD
:1020340040030220BFE56875F00A84FF7E00900526
:1020440077120048E0F55B755A00AE5AAF5B90001A
:1020540092E01270FE74648E048F05FF1270EE8C91
:102064005C8D5D9000EFE004C395448C068D0712EF
:1020740070FE9000EFE08E048F05FF1270EE8C5C12
:102084008D5D90087FE0FEA3E0FFEF2DFDEE3CFCAC
:1020940090087FECF0A3EDF09000DDE0B4021A901C
:1020A4000881E0FEA3E0FFAA5CAB5DEF2BFBEE3AF8
:1020B400FA900881EAF0A3EBF080569000EFE00478
:1020C400C39544854CF0A4FFAEF09000EFE08E047D
:1020D4008F05FF1270EE8C5C8D5D90087FE0FEA38F
:1020E400E0FFEF2DFDEE3CFC90087FECF0A3EDF05B
:1020F4009000DDE0B4021A900881E0FEA3E0FFAA9C
:102104005CAB5DEF2BFBEE3AFA900881EAF0A3EBAF
:10211400F005449000EFE0C39544500375440090EB
:10212400009CE05401601B900090E0A852B800129B
:10213400D39553400DA204B3B35007E560C394CCC8
:102144004002806090008EE075F003A4FFAEF0E5DD
:10215400412FFF50010E74032FFF50010EE560BEA6
:102164000042D39F403E754501A231403790008F15
:10217400E075F05EA4FFAEF074058E048F05FF12C7
:1021840070EE8C5C8D5D124ABD90087FE0FEA3E08A
:10219400FF90008FE02FFF50010E90087FEEF0A318
:1021A400EFF0D231E560C395415002C23185604100
:1021B400E54570030222BD9000F0E0C3954550034D
:1021C4000222AF9000FFE0C394024003022259E5CB
:1021D4006875F00A84FF7E00900577120048E0F5E8
:1021E4005B755A00AE5AAF5B90008FE01270FE74BC
:1021F400648E048F05FF1270EE8C5C8D5D9000F090
:10220400E004C395458C068D071270FE9000F0E043
:102214008E048F05FF1270EE8C5C8D5D90087FE05C
:10222400FEA3E0FFEF2DFDEE3CFC90087FECF0A355
:10223400EDF09000DDE0B4021A900881E0FEA3E026
:10224400FFAA5CAB5DEF2BFBEE3AFA900881EAF053
:10225400A3EBF080569000F0E004C39545854DF063
:10226400A4FFAEF09000F0E08E048F05FF1270EE34
:102274008C5C8D5D90087FE0FEA3E0FFEF2DFDEE0A
:102284003CFC90087FECF0A3EDF09000DDE0B4029C
:102294001A900881E0FEA3E0FFAA5CAB5DEF2BFB84
:1022A400EE3AFA900881EAF0A3EBF005459000F0CD
:1022B400E0C39545500375450090087FE0FEA3E018
:1022C400FF9000A1E0BE00039F500D9000A1E0909C
:1022D400087FF8E4F0E8A3F09000DDE0B402129087
:1022E4000881E0FEA3E0FF9000A1E0BE00059F404E
:1022F40002800D9000A1E0900881F8E4F0E8A3F0DA
:10230400229000DDE0B401028003022453A204B34E
:10231400500302243A9000A8E0B4017A90087FE0C8
:10232400FEA3E0FFAC52AD53120003743C8E048F45
:1023340005FF1270EE9000B8E0BC00159D401290AD
:10234400087FE0FEA3E0FF9000BAE0BE00039F50C8
:1023540002D20390087FE0FEA3E0FFAC52AD53121B
:102364000003743C8E048F05FF1270EE9000B8E0F9
:10237400C3940ABC001AD39D401690087FE0FEA3C4
:10238400E0FF9000BAE0C39405BE0004D39F50025E
:102394008002C203807A90087FE0FEA3E0FFAC5283
:1023A400AD5312000374788E048F05FF1270EE9003
:1023B40000B8E0BC00159D401290087FE0FEA3E049
:1023C400FF9000BAE0BE00039F5004D20380419006
:1023D400087FE0FEA3E0FFAC52AD53120003747813
:1023E4008E048F05FF1270EE9000B8E0C3940ABC0F
:1023F400001AD39D401690087FE0FEA3E0FF9000F2
:10240400BAE0C39405BE0004D39F50028002C20305
:10241400A203B3402190087FE0FEA3E0FF9000B93F
:10242400E01270FE74648E048F05FF1270EE900843
:102434007FECF0A3EDF0A203B3400CA23540067488
:1024440024900043F0D235A2034002C2358002C278
:102454000390003EE06006A204B3B34002801990EA
:10246400087FE0FEA3E0FF90003EE02FFF50010E46
:1024740090087FEEF0A3EFF0A201B34006A202B3EE
:10248400B35009900016E4F0A3F0802D90087FE08B
:10249400FEA3E0FF7400D39F74019E401190087F57
:1024A400E0F8A3E0900016C8F0A3C8F0800B74FF16
:1024B400900016F8E4F0E8A3F09000BFE0C39404A1
:1024C400400C9008E1E0C3940240030225AD900063
:1024D400A8E0B4014790087FE0FEA3E0FF745E1219
:1024E40070FE74058E048F05FF1270EE90087FEC69
:1024F400F0A3EDF09000DDE0B4021F900881E0FE4F
:10250400A3E0FF745E1270FE74058E048F05FF1243
:1025140070EE900881ECF0A3EDF0804590087FE028
:10252400FEA3E0FF745E1270FE740A8E048F05FF32
:102534001270EE90087FECF0A3EDF09000DDE0B4B3
:10254400021F900881E0FEA3E0FF745E1270FE7427
:102554000A8E048F05FF1270EE900881ECF0A3ED53
:10256400F090087FE0FEA3E0FF7402BE000CD39F4E
:102574004008752A02752900800A90087FE0F52931
:10258400A3E0F52A900881E0FEA3E0FF7402BE00F8
:102594000CD39F4008752E02752D00800A90088187
:1025A400E0F52DA3E0F52E804690087FE0FEA3E041
:1025B400FF7401BE000CD39F4008752A01752900E1
:1025C400800A90087FE0F529A3E0F52A900881E0CD
:1025D400FEA3E0FF7401BE000CD39F4008752E01DA
:1025E400752D00800A900881E0F52DA3E0F52E906A
:1025F4000014E529F0A3E52AF0A238B34009C2018A
:10260400900016E4F0A3F022900042E090037712C9
:10261400712FE0F542754364900042E0FE9000B3F0
:10262400E0D39E4037E56075F00884FF7E008F3864
:10263400E56075F00884ADF07C008D3B754008754D
:102644005A03755B96E538C3941F50051211C58073
:102654000690042CE0F5388538438035E56075F044
:102664000884FF7E008F38E56075F00884ADF07C47
:10267400008D3B754008755A03755BB6E538C39405
:102684001F50051211C5800690044CE0F5388538BA
:1026940043229000E9E0F53D754011755A04755BDD
:1026A40000AE52AF53E53D75F00FA4FDACF0EDD391
:1026B4009FEC9E4021E53D8E048F05FF1270EEEDE8
:1026C40075F010A4FFAEF0E56075F01184FD7C0098
:1026D400ED2FF53E800EE56075F01184FF7E00EF6E
:1026E40024F0F53E853E38E56075F01184AFF07E48
:1026F400008F3B1211C585383FAE52AF539000E9AD
:10270400E075F00FA4FDACF0EDD39FEC9E4028756E
:102714005A04755B10853E381211C5853F398538DA
:102724003AAE52AF53E53D8E048F05FF1271198DF9
:102734003B853D3C12123F8538427543642290002C
:10274400E9E0F53D754011755A04755B00AE52AF72
:1027540053E53D75F00FA4FDACF0EDD39FEC9E4026
:1027640021E53D8E048F05FF1270EEED75F010A487
:10277400FFAEF0E56275F01184FD7C00ED2FF53EAF
:10278400800EE56275F01184FF7E00EF24F0F53EC3
:10279400853E38E56275F01184AFF07E008F3B1200
:1027A40011C585383FAE52AF539000E9E075F00F84
:1027B400A4FDACF0EDD39FEC9E4028755A04755BE4
:1027C40010853E381211C5853F3985383AAE52AF6F
:1027D40053E53D8E048F05FF1271198D3B853D3CF9
:1027E40012123F8538427543649000E4E0B40479E2
:1027F400900042E0FE9000B3E0D39E4037E5607560
:10280400F00884FF7E008F38E56075F00884ADF031
:102814007C008D3B754008755A03755B96E538C39B
:10282400941F50051211C5800690042CE0F53885DC
:1028340038438035E56075F00884FF7E008F38E505
:102844006075F00884ADF07C008D3B754008755AC6
:1028540003755BB6E538C3941F50051211C5800695
:1028640090044CE0F5388538432290007DE0B401B3
:102874003BE56875F00A84FF7E008F38E56875F0E3
:102884000A84ADF07C008D3B75400A755A05755B72
:1028940012E538C3941150051211C5800690059AAB
:1028A400E0F538E5432538C39464F54390007EE0B1
:1028B400B4013BE56975F00A84FF7E008F38E56951
:1028C40075F00A84ADF07C008D3B75400A755A059D
:1028D400755B7EE538C3941150051211C5800690CE
:1028E4000606E0F538E5432538C39464F543E5422C
:1028F4002543F537900085E0B402109008D9E0250F
:1029040037FE9000D9E0F4042EF5379000DCE0D3D4
:1029140094014040E56CC394E7501D74E7C3956C83
:10292400FE9008DBE08E00F5F0E884FF7E008F382F
:10293400E5372538F537801CE56CC394E7FE90082D
:10294400DBE08E00F5F0E884FF7E008F38E537C3C6
:102954009538F537A2044006E5422464F537E53797
:10296400D394644009E537C39464F537800375371D
:10297400009000B5E0C3953750069000B5E0F537F8
:1029840022D201900065E0A852B800049553503E4D
:10299400900065E0A852B800049553500375370FB2
:1029A400900065E004A852B80004955350037537AD
:1029B40007900065E02402A852B800049553500221
:1029C400C201900065E060067409900043F0C230D3
:1029D4007E017F009000BBE01270FE9000CAE08E82
:1029E400048F05FF1270EEE560BC000CD39D400817
:1029F400D238740A900043F090007DE0B40109904D
:102A040000BCE0C39568400280159000CEE0A85257
:102A1400B8000495535002C201740B900043F09027
:102A2400007DE0B40107E568C394644002801D9012
:102A34000114E0600D900114E0A852B8000695530B
:102A440040028008C201740B900043F0A2014003CD
:102A5400753700C2379000FDE0B401149000FEE029
:102A6400A852B8000495535007E560C3956140022D
:102A7400802A9000A6E0D3941D400B9000A6E0C3EA
:102A8400941EF5378003753700A2344008741590FE
:102A94000043F0D237D234D232022B7FC232C23456
:102AA400900085E0B40306A22AB3B34003022B7F4F
:102AB4009008DDE0C39405A852B80004955350066D
:102AC4009008E4E06002801F9000A6E0D3941D40CB
:102AD4000B9000A6E0C3941EF5378003753700748D
:102AE4000C900043F0D2379008DDE0A852B80004FF
:102AF400955350069008E4E07002801F9000A6E011
:102B0400D3941D400B9000A6E0C3941EF5378003B8
:102B1400753700740C900043F0D2379008DDE0A8BC
:102B240052B80004955350319000C4E0B40228D246
:102B3400309008E3E0FE9008E4E0D39E500690084D
:102B4400E4E0700280099008E3E4F0C2308006906B
:102B540008E3E004F08002C2019008DDE02405A847
:102B640052B80004955350139000C4E0B4020A9084
:102B740008E4E07002D2308002C201A22FB34027E1
:102B84009000A6E0D3941D400B9000A6E0C3941ED1
:102B9400F5378003753700A2334006741090004364
:102BA400F0D233D2378002C23385376D9000A6E06D
:102BB400D3941D4018900074E02537FE900042E045
:102BC40075F01E84FC7F00EE2CF5378037A237B3F6
:102BD4004016900074E0FE900042E075F01E84FC04
:102BE4007F00EE2CF537801C900076E02537FE90B0
:102BF4000074E02EFE900042E075F01E84FC7F001D
:102C0400EE2CF537A238B34005D230756D00229012
:102C14000042E075F00584FF7E008F38900042E0AA
:102C240075F00584ADF07C008D3B754005755A0345
:102C3400755BD69000C8E01475F00584FF7E00E54E
:102C440038BE00039F50051211C5800BE53890046F
:102C54004D12712FE0F538E5389008DCF09008DC6F
:102C6400E0FE9000B7E0C39E50089000B7E09008E3
:102C7400DCF09000A6E0D3941D401E9008DCE0FE3A
:102C8400900074E02EFE900042E075F01E84FC7FFC
:102C940000EE2C9008DCF0803FA237B3401890007F
:102CA40074E0FE900042E075F01E84FC7F00EE2C80
:102CB4009008DCF080229008DCE0FE900076E02EA4
:102CC400FE900074E02EFE900042E075F01E84FC3D
:102CD4007F00EE2C9008DCF02290007DE0B40136F9
:102CE400E56875F00A84FF7E00900577120048E0DD
:102CF400F547E547D394644010E547C3946475F001
:102D04000F84FF7E008F47800375470090009AE090
:102D14002547F547800690009AE0F54722E5687557
:102D2400F00A84FF7E00900577120048E0C394699E
:102D34004007E568D3946440559000E4E0C39403ED
:102D44005026900879E0FEA3E0FF7404120039E5F0
:102D5400601270FE740F8E048F05FF1270EE9008DF
:102D640077ECF0A3EDF08024900879E0FEA3E0FF77
:102D74007404120039E5621270FE740F8E048F051C
:102D8400FF1270EE900877ECF0A3EDF0800F90083E
:102D940079E0F8A3E0900877C8F0A3C8F0A2044053
:102DA4001A900879E0FEA3E0FF74031270FE740128
:102DB400120039900877EEF0A3EFF090008DE0B4A4
:102DC4000262E56BC3944175F00584FF7E008F3881
:102DD400E56B75F00584ADF07C008D3B75400575A1
:102DE4005A06755B14E538C3941750051211C58053
:102DF4000690069EE0F538900877E0FEA3E0FF74A5
:102E04000A8E048F05FF1270EEE5388C068D0712CA
:102E140070FE740A8E048F05FF1270EE900877EC32
:102E2400F0A3EDF0900877E0FEA3E0FF90087DE0CA
:102E3400FCA3E0FDEDD39FEC9E400F90087DE0F8ED
:102E4400A3E0900877C8F0A3C8F022E50875F00461
:102E5400A4FFAEF09006BA120048E0903CE8F828CF
:102E64002873804C85537480479000CAE08560F0D5
:102E7400A4FFAEF074081200398F74803385627435
:102E8400802E85687480298569748024856A74809D
:102E94001F856B74801A856C748015856774801027
:102EA400856674800B856D748006900017E0F57458
:103CE800022E66022E68022E6D022E81022E860298
:103CF8002E8B022E90022E95022E9A022E9F022EB5
:073D0800A4022EA9022EAE59
:102EB400E50875F004A4FFAEF09006BB120048E5E7
:102EC4000875F004A4FFAEF0E0FC9006BC120048C4
:102ED400ECFEE0FFEEC39F4003022FBCE50875F053
:102EE40004A4FFAEF09006BA120048E0B40441E531
:102EF4000875F004A4FFAEF09006BC120048E0C3CD
:102F04009574500AE508F50CD39239123E8DE50804
:102F140075F004A4FFAEF09006BB120048E0D39510
:102F240074400AE508F50CC39239123E8D022FBA9B
:102F3400E50875F004A4FFAEF09006BB120048E06B
:102F4400C395745015E50875F004A4FFAEF090061F
:102F5400BC120048E0D395745002800AE508F50CD1
:102F6400D39239123E8DE50875F004A4FFAEF090BB
:102F740006BB120048E0D395745015E50875F004BB
:102F8400A4FFAEF09006BC120048E0C39574500A4A
:102F9400E508F50CC39239123E8D9006C2E0B401E7
:102FA400099000D6E0D395625002800A7402F50CB1
:102FB400C39239123E8D806AE50875F004A4FFAE11
:102FC400F09006BB120048E0D395744015E50875EF
:102FD400F004A4FFAEF09006BC120048E0C3957460
:102FE4004002800AE508F50CC39239123E8DE508CB
:102FF40075F004A4FFAEF09006BB120048E0C39540
:10300400744015E50875F004A4FFAEF09006BC12F8
:103014000048E0D39574400AE508F50CD3923912C0
:103024003E8D22AE2FAF3074C9BE000CD39F400832
:10303400782F127151023141753001752F00AE5253
:10304400AF53E547BE000DD39F40099000ACE0D3D9
:10305400954840028023754800E547C39553F574AD
:103064009000AFE0D395464008E5462574F54680C8
:10307400069000AFE0F54680020548900088E0D352
:103084009562401CE560C395614015AE52AF53E5AF
:1030940047BE00039F50099000ADE0D3954940021C
:1030A400806E9008DEE0A852B80004955350037572
:1030B4004B009008DEE0A852B8000BD395534006AD
:1030C400E5539008DEF0E54B7041E553C39547F5B1
:1030D40074E574D3940540037574059000AEE0C3A1
:1030E40095465007E574C3954640028009E546C3FA
:1030F4009574F54680069000AEE0F5469000AEE08B
:10310400D3954640069000AEE0F54675490080022E
:103114000549E54B7016900088E0C39562500DE5B3
:10312400472405A852B8000695534002800F90002A
:103134009BE0F546754B0174789008DEF022AE2FC3
:10314400AF3074E9D39F74039E4008782F127151F5
:103154000232FB753001752F00754632A22B403DBB
:10316400E54875F00284AFF07E00EF4E70057546B9
:1031740019800375463290009BE075F002A4FFAEFF
:10318400F0E548BE0006D39F4002D22B0548754B9C
:103194000374789008DEF0754A000232E2AE52AF52
:1031A40053E5476F4E70030232E2E547BE000DD38C
:1031B4009F40099000ACE0D395484002800F7548C9
:1031C40000E54BC394035003754619800DE547C3CE
:1031D4009553F574E5482574F548900088E0D39537
:1031E40062400E9008DEE0A852B80007D395534021
:1031F40002800C054A90009BE0B54A03754B00E53C
:103204004BB40306A204B3B34002800A054AE54A5C
:10321400B43C03754B02E54BB402299008DEE0A8E8
:1032240052B8000ED395534009E5539008DEF0756B
:103234004A00900088E0C395625009754A0074788A
:103244009008DEF0E54B705A900088E0D395624018
:103254001CE560C395614015AE52AF53E547BE000F
:10326400039F50099000ADE0D39549400280087552
:10327400490075464B8028E553C39547F574E574BA
:10328400D394054003757405900088E0D39562409B
:1032940008E5492574F5498006E5492406F549758C
:1032A4004A00E54B7016900088E0C39562500DE526
:1032B400472405A852B80006955340028003754B75
:1032C40001E54BB40118754619054A90009BE0B519
:1032D4004A06754B02754A0074789008DEF0A20223
:1032E400B34003754632E54675F00AA4FFAEF0908C
:1032F4000883EEF0A3EFF022E570903D0FF8282844
:1033040073023CA8900080E0700302362C9000B653
:10331400E0B4010280030234BF900040E0655F60C6
:1033240009E553455260030234BC7E017F00E5BECB
:103334001270FEE5BD2FFF50010E8E5A8F5B900177
:103344001BE075F010A4FDACF08C5C8D5DEFD39D9B
:10335400EE9C40091271498E5A8F5B8006755B00A2
:10336400755A00AE5AAF5B740E1270FE9000ABE05B
:103374008E048F05FF1270EE900887ECF0A3EDF039
:10338400E56C600FE56CC394FE50089000DCE064CB
:1033940002600280649000CAE0B40B1F900887E0CA
:1033A400FEA3E0FF74E71270FEE56C8E048F05FF48
:1033B4001270EE900887ECF0A3EDF09000CAE0D311
:1033C400940B40089000B2E064046002802B9008E3
:1033D40087E0FEA3E0FF90088BE0FCA3E0FDEFD3C1
:1033E4009DEE9C400D127149900887EEF0A3EFF01A
:1033F4008007900887E4F0A3F0900887E0FEA3E03C
:10340400FFEFD39400EE94014008D2387426900064
:1034140043F0A238B3B3502C7E057F009000CAE07D
:103424008E048F05FF1270EE900887E0FEA3E0FF84
:10343400EFC39DEE9C400FAC52AD53740FBC00041F
:10344400D39D50028002C238900080E0B4022790DD
:103454000889E0FEA3E0FF900887E0FCA3E0FDEF0D
:103464002DFDEE3CFC74018C068D0712003990088A
:1034740087EEF0A3EFF0900887E0FEA3E0FF90084A
:1034840089E0FCA3E0FDEDD39FEC9E4004D22E80A6
:1034940002B22E900887E0F8A3E0900889C8F0A350
:1034A400C8F09000B2E064016006A22EB3B34002FB
:1034B4008006900888E0F56002362AD22E7E017FCD
:1034C40000E5BE1270FEE5BD2FFF50010E8E5A8F2F
:1034D4005B90011BE075F010A4FDACF08C5C8D5D7D
:1034E400EFD39DEE9C40091271498E5A8F5B800682
:1034F400755B00755A00AE5AAF5B740E1270FE9085
:1035040000ABE08E048F05FF1270EE900887ECF09C
:10351400A3EDF0E56C600FE56CC394FE50089000D9
:10352400DCE06402600280649000CAE0B40B1F9087
:103534000887E0FEA3E0FF74E71270FEE56C8E04DA
:103544008F05FF1270EE900887ECF0A3EDF0900069
:10355400CAE0D3940B40089000B2E0640460028097
:103564002B900887E0FEA3E0FF90088BE0FCA3E02B
:10357400FDEFD39DEE9C400D127149900887EEF04B
:10358400A3EFF08007900887E4F0A3F0900887E0A9
:10359400FEA3E0FFEFD39400EE94014008D2387408
:1035A40026900043F0A238B3B3502C7E057F0090E0
:1035B40000CAE08E048F05FF1270EE900887E0FECB
:1035C400A3E0FFEFC39DEE9C400FAC52AD53740FCC
:1035D400BC0004D39D50028002C238900080E0B445
:1035E4000227900889E0FEA3E0FF900887E0FCA38F
:1035F400E0FDEF2DFDEE3CFC74018C068D071200FE
:1036040039900887EEF0A3EFF0900887E0F8A3E084
:10361400900889C8F0A3C8F09000B2E06401600685
:10362400900888E0F560800375600090007CE0708D
:10363400067570030232FC75BB18023CA8023CA854
:1036440090007CE070030237B57E017F00E5BE1276
:1036540070FEE5BD2FFF50010E8E5A8F5B9000C2A5
:10366400E0B4010F7E0F7FFFAC5AAD5B1271498E3F
:103674005A8F5B9000E7E0B40245AE5AAF5B90000E
:1036840020E0FCA3E0FDEDD39FEC9E400A900020D7
:10369400E55AF0A3E55BF0AE5AAF5B900022E0FC84
:1036A400A3E0FDEFD39DEE9C400A900022E55AF082
:1036B400A3E55BF0AE5AAF5B74041200398F6290DD
:1036C40000E7E0704CAE5AAF5B900020E0FCA3E052
:1036D400FDEFD39DEE9C40091271498E5A8F5B8099
:1036E40006755B00755A00AE5AAF5B74101270FE1B
:1036F4009000E6E08E048F05FF1270EE8C5A8D5B0D
:1037040074FFBC0009D39D4005855B62800375622C
:10371400FE9000B2E0B4010280030237B3A204B306
:10372400B3500E900086E0A852B80005D3955350CC
:103734000280719000C3E08562F0A4FFAEF074646F
:103744008E048F05FF1270EE8C5A8D5BE56C60164B
:10375400E56CC394FE500F9000DCE0B402089000C6
:10376400CAE0640B60028017AE5AAF5B74E7127054
:10377400FEE56C8E048F05FF1270EE8C5A8D5BAEE5
:103784005AAF5B900887E0FCA3E0FDEDD39FEC9E6D
:103794004005855B60800BA22EB34006900888E04C
:1037A400F560800BA22EB34006900888E0F5608097
:1037B4000375620090007FE070067570050232FCAC
:1037C40075BB19023CA8023CA890007FE07003027C
:1037D400389CE55FD3955E400302389A90001EE062
:1037E400FEA3E0FFE56612714190001EEEF0A3EF28
:1037F400F09000ECE0B402247E017F00E5BE12707C
:10380400FEE5BD2FFF50010E8F048E057E0F7FFF56
:10381400CDCCCD1271498E5A8F5B80147E017F000E
:10382400E5BE1270FEE5BD2FFF50010E8E5A8F5B70
:103834009000ECE07017AE5AAF5B740A1270FE741D
:10384400518E048F05FF1270EE8D668019AE5AAF4B
:103854005B740A1270FE8F048E057E017F95CDCCB9
:10386400CD126FEC8F66E566D3946440037566648D
:1038740090001EE0FEA3E0FFE5662FFF50010E90CE
:10388400001EEEF0A3EFF0900083E0048E048F0599
:10389400FF1270EE8D6680037566329000CFE07083
:1038A400067570070232FC75BB13023CA8023CA8E3
:1038B4009000CFE0604A7E017F00E5BE1270FEE515
:1038C400BD2FFF50010E8E5A8F5B74041200398F86
:1038D400679000D1E08567F0A4FDACF07464FF123A
:1038E40070EE8D679000D0E08567F0A4FFAEF074B1
:1038F400FF8E048F05FF1270EEED900064F08003DC
:1039040075670090007DE070067570090232FC75E1
:10391400BB17023CA8023CA890007DE0B4010280E1
:10392400030239B07E017F00E5BE1270FEE5BD2FB3
:10393400FF50010E8E5A8F5B9008DFE060199008EB
:10394400DFE014906ADE12008CE493FC740193FDB2
:10395400EDC39FEC9E400280069008DFE014F090D7
:1039640008DFE0C394B3501DAE5AAF5B9008DFE0AC
:1039740004906ADE12008CE493FC740193FDEFC39F
:103984009DEE9C400280069008DFE004F09008DF82
:10399400E0FE9000A3E08E0088F0A4FFAEF0746413
:1039A4008E048F05FF1270EE8D6880037568009099
:1039B400007EE0700675700B0232FC75BB16023C8B
:1039C400A8023CA890007EE0B401028003023A5CA5
:1039D4007E017F00E5BE1270FEE5BD2FFF50010E93
:1039E4008E5A8F5B9008E0E060199008E0E0149034
:1039F4006C4812008CE493FC740193FDEDC39FECBE
:103A04009E400280069008E0E014F09008E0E0C3D5
:103A140094B3501DAE5AAF5B9008E0E004906C483C
:103A240012008CE493FC740193FDEFC39DEE9C4063
:103A34000280069008E0E004F09008E0E0FE9000C8
:103A4400A9E08E0088F0A4FFAEF074648E048F05A4
:103A5400FF1270EE8D69800375690075BB1F023C0F
:103A6400A8023CA87E017F00E5BE1270FEE5BD2FD2
:103A7400FF50010E8E5A8F5B74091270FE74E68E2D
:103A8400048F05FF1270EE8D6B900085E070067553
:103A9400700F0232FC75BB15023CA8023CA89000D2
:103AA40085E07003023BF37E017F00E5BE1270FEE9
:103AB400E5BD2FFF50010E8E5A8F5B74041200393E
:103AC4008F6A900085E0B401159000D9E0856AF012
:103AD400A4FFAEF07407120039EF9008DAF09000FA
:103AE40085E0B402159000D9E0856AF0A4FFAEF039
:103AF4007407120039EF9008D9F0900085E0B40300
:103B0400028003023BD69000C6E07052E56AC3947B
:103B140019500FD22A9000A5E09008DDF09008E239
:103B2400E4F0E56AD394644004A22A4002802D9014
:103B340008E2E004F09008E2E0FE900118E0B50627
:103B44000B9008DDE004F09008E2E4F09008DDE07A
:103B540064966006900118E07002C22A80639000A7
:103B6400A5E070349000D9E0856AF0A4FFAEF0744B
:103B7400FF8E048F05FF1270EEED9008DDF0AE525B
:103B8400AF53741EBE0006D39F4002D22AE562D30F
:103B940094E54002C22A8029E56AC3940A500DAE16
:103BA40052AF53741EBE0004D39F50028002D22A27
:103BB400E562D394E54002C22A9000A5E09008DDB6
:103BC400F09008DDE0C39405500674059008DDF01C
:103BD400C22F900085E0B40414E56AC3941950021E
:103BE400D22FE56AD394324002C22FC22A800375D1
:103BF4006A009000DCE070067570110232FC75BB3F
:103C040014023CA8023CA89000DCE07003023C953E
:103C14007E017F00E5BE1270FEE5BD2FFF50010E50
:103C24008E5A8F5B90011CE075F010A4FDACF08CF3
:103C34005C8D5DEFD39DEE9C40091271498E5A8FC5
:103C44005B8006755B00755A00AE5AAF5B740E124A
:103C540070FE9000E3E08E048F05FF1270EE8C5C22
:103C64008D5D74FFBC00039D5005756CFF8003855A
:103C74005D6CE56C75F00BA4FFAEF09000CAE08EAD
:103C8400048F05FF1270EE90088BECF0A3EDF0802A
:103C940003756C00900080E0600575BB1A800375A5
:043CA400BB188000C9
:103D0F000233050233080236410236440237CA0233
:103D1F0037CD0238B10238B402391902391C0239D1
:103D2F00C50239C8023A65023A68023A9F023AA2BE
:093D3F00023C08023C0B023CA806
:103CA800E57075F00284AFF07E00EF4E7002D2EC42
:033CB80005702272
:09712F002582F58250020583223D
:0F008C0025E050020583258250020583F582226C
:1070CD00EF2F500205832582F582E5833E2EF58351
:0170DD002290
:10714100CFC39FFF50011E22C3EF9DFFEE9CFE2285
:087151000806B6000218062230
:0D710C00A3E004F07006127125E004F022EB
:0E003900048007C3CE13CECF13CFD5E0F6223E
:106FEC00BC000FBE0008ED8FF084FFADF022E4FE74
:106FFC00FF22BE000DEF60FE54F0606F20E703022D
:10700C0070A2EAC0E0EBC0E078017A0075F001EE06
:10701C0020E710EF25E0FFEE33FE0AC5F023C5F0A4
:10702C0030E7F0EA5407F9096A7A007B006001083E
:10703C00C3EC9E40167004ED9F4010ED9FFDEC9E3E
:10704C00FCE5F0CA4ACA03F5F08005E5F003F5F05B
:10705C00C3EE13FEEF13FFD9D77908CACBCAD8D029
:10706C00EAFEEBFFD0E0FBD0E0FA22EC8FF084FCE0
:10707C00ED54F045F0C48FF084FEEDC454F045F0AF
:10708C00C48FF084FDEEC4FE54F02DFFEE540F3C83
:10709C00FEADF07C0022790078008FF0EC7E0820A9
:1070AC00E70DC3CD33CD33C933C9C833C8DEF08443
:1070BC0049F9E5F08FF0BE00E6FD7C00E9FFE8FE43
:0170CC0022A1
:0E70FE00F88FF0A4FFE5F0CE88F0A42EFE225D
:10000300EF8DF0A4F9A8F0EF8CF0A428F8EE8DF0B2
:06001300A428FEE9FF2213
:1070DE00600D782B0270E8007830D8FED5E0F822EB
:1070EE00EEC0E07E00126FECEFFDEEFCD0E0FE2273
:0C711900EEC0E07E00126FECD0E0FE2221
:03001B0002001EC2
:0300530002005652
:03009B00020071EF
:0300000002713852
:0971380075817675D000024C2629
:0B004800E5822FF582E5833EF5832260
:0A7125000582D5820215831582222F
:10001E00C0E0C0F0C083C082C0D075D000124B903B
:0B002E00D0D0D082D083D0F0D0E032E0
:10005600C0E0C0F0C083C082C0D075D000124B9300
:10006600D0D0D082D083D0F0D0E032C0E0C0F0C093
:1000760083C082C0D075D000124BE8D0D0D082D0D9
:0600860083D0F0D0E0324F
:00000001FF
